:020000040800F2
:10500000F81B0020D5500008E98A0008C581000877
:105010000000000000000000000000000000000090
:105020000000000000000000000000004999000896
:105030000000000000000000C5920008859A0008EA
:10504000E7500008E7500008E7500008E750000864
:10505000E7500008D95C0008E7500008E750000856
:1050600000000000E7500008015C0008E75000085D
:10507000E7500008D986000800000000E75000084B
:1050800000000000E75000080000000000000000E1
:10509000E750000800000000E7500008E750000853
:1050A000E7500008E7500008E750000815A5000881
:1050B000E7500008E7500008000000000000000072
:1050C0000348854600F0E8FC0048004795B8000812
:1050D000F81B00200448804704480047FEE7FEE72D
:1050E000FEE7FEE7FEE7FEE7219B0008C15000084F
:1050F00030B50B46014600202022012409E00D4670
:10510000D5409D4205D31D469540491B25469540F7
:1051100040191546521E002DF1DC30BDF0B51FB40C
:105120000646002082B005464024019100901BE015
:10513000019922460F46304600F098FB049A059BE1
:10514000801A994110D310461946224600F07EFB82
:10515000361A8F410197224601200021009F00F05E
:1051600075FB38184D4100902046641E0028DFDC96
:10517000019B00982946324607B0F0BD03460B4319
:105180009B0703D009E008C9121F08C0042AFAD2FD
:1051900003E00B780370401C491C521EF9D2704783
:1051A000D2B201E00270401C491EFBD270470022BF
:1051B000F6E710B513460A4604461946FFF7F0FF16
:1051C000204610BD30B504460020034600E05B1CBD
:1051D000934203D2E05CCD5C401BF8D030BDF8B503
:1051E00002464A40D40F42004B0052085B089A42E4
:1051F00002D20246084611464A0023D0C30D4A0097
:10520000DDB2120EAD1A202D35DA49020126490A07
:10521000F6058A19002C00D0524220214F1B11465E
:10522000B9402A411018C20D9A4221D0002C17D043
:10523000012D08DCDA05801AD20F8019D207DBB203
:1052400000F040FBF8BDDA05801A012340001B0680
:10525000C01880185A428018CA0F1043490007E04E
:105260004908C2071143DA05801A801940088018DE
:1052700000F020FBF8BD61000122511A001BF7E786
:105280000122D2075140AAE70122D2075040A6E7E7
:1052900070B502464A40D50F40004A00ED0740086D
:1052A0005208002814D0002A12D0C40DD30D410298
:1052B0000120C0055202490A520AE41A09181218BC
:1052C0007D34914201D3641C00E04900002C01DAD6
:1052D000002070BD0023914201D3891A0343400886
:1052E00049000028F7D100290AD0914202D10121BA
:1052F000C90705E0914201D2012101E00121C94322
:10530000E005C018401900F0D5FA70BD420005D084
:105310004200120E52428A4201DB00207047C9054A
:1053200008187047F0B507460846584087B0C00FC8
:10533000049048000E46590040084908BC1A8841AC
:1053400005D2384631461E4617460B4602465800DF
:10535000400810434CD0300D039040055900400DDB
:10536000490D0590401A0290402872DA1803012175
:10537000000B09050843019004980092002805D00D
:1053800001995242002088410092019002984021E8
:105390000A1A0199009800F059FA05460C466B4626
:1053A00007CB00F074FAC0197141039A0E0D002367
:1053B000D71756401A467A40164344D0049A002A1A
:1053C0002DD0029A012A039A15DC1205C01A9141C8
:1053D00001263605001C7141D20F059ED2070093AD
:1053E000019202962A46234600F0B2FA07B0F0BDB9
:1053F00038463146FAE71605224A0F46B218C01A57
:10540000B74101210905001C4F4100187F41114699
:1054100018187941E20F10436D19644113E0E20757
:105420006D0815436408C2071443039A0126120548
:10543000C01A91413605001C7141CE074008304327
:105440004908C01851412A46234600F074FACDE7B6
:10545000FFE7049801224000C117121A00238B4174
:1054600004983146C417381AA141EEE730B401243C
:10547000E407634030BC55E730B40124E4076140E1
:1054800030BC4FE70000E0FFF0B51FB488B00B99C7
:105490000998002448400999C00F4900490809911A
:1054A000C0070B990090490049080B910999089889
:1054B000A64608431CD00B990A98084318D00998AF
:1054C00001244000420D4800410D099824050003C5
:1054D000000B204309900B980003000B20430B9016
:1054E00050181C494018002201901446104605E04F
:1054F000002001460DB0F0BD032801DA034600E0AC
:1055000003239C46C11A0AAE0AE05F0008ADED5BBA
:105510004F00F75B7D430027AA187C41491C5B1EA6
:105520006145F2DD410004AB5A522104120C0A43DA
:10553000240C401C0828DFDB01980290009970467B
:1055400001910090059B049A0799069800F000FAD3
:10555000D0E700000DFCFFFFF0B50C465C4085B0C5
:10556000E40FE40703944C000026640859009446B5
:10557000490802460296224321D062460A431ED0C1
:105580006200570D4A000E032303550D0124024605
:105590002C492405781B1B0B360B4018234326434C
:1055A000614600901C46501AB44103D30098401C39
:1055B000009002E0921800985B41002803DA002076
:1055C000014605B0F0BD00200121090507468646C9
:1055D00011E064461D46141BB54106D36546521BB7
:1055E000B341744607430C43A646CD07400849081B
:1055F000284392185B4105460D43EAD110461843F3
:1056000013D06046194650407140084306D06046AA
:10561000101AB34106D20122002306E00022012322
:10562000DB0702E00122D2435310009874460105C3
:10563000381C6141029C039D0019694100F07BF90F
:10564000BFE70000FD03000070B54B005B0803439B
:105650000BD04B005C0D002633466542B341D41796
:10566000AD1AA34102DB0020014670BD12053018BF
:10567000514170BDC217C10F504010B54018CA0744
:105680009623002100F01EF910BD10B500229623CC
:10569000114600F017F910BD0EB5C217C10F5040EA
:1056A000CA0740180021054B0293019200910A4657
:1056B0000B4600F04DF903B000BD000033040000BC
:1056C0000EB505490291002100910A460B46019151
:1056D00000F03EF903B000BD330400004100400279
:1056E0000122400AD205090E80187F2901DA002024
:1056F0007047962903DC9622511AC84070479639A4
:105700008840704770B5CD0F4A0009030123090B8B
:105710001B0519430B4BED070024520D9A4201DA89
:10572000002070BD074B34339A4203DC9A1A00F014
:105730009DF802E00449511888402C43F1D04042C2
:1057400070BD0000FF030000CDFBFFFF4A0009030E
:105750000123090B1B051943094B10B5520D9A4241
:1057600001DA002010BD064B34339A4203DC9A1A4A
:1057700000F07CF810BD03495118884010BD0000AE
:10578000FF030000CDFBFFFFC20FD207400040081F
:105790000BD0C10D0723DB01C91840020905400ADF
:1057A0001143C2084007114370470020014670476B
:1057B00010B5002904DB0124E40740428C41214656
:1057C000002B04DB1C460123DB075242A3418B4222
:1057D00000D1824210BD000010B5002904DB012475
:1057E000E40740428C412146002B04DB1C46012388
:1057F000DB075242A341994200D1904210BD000004
:10580000CB0FDB07490010B5490802460A4307D011
:105810000A0D07240903E401090B121B002A01DC0D
:10582000002010BDC900440F0C43C100E018D20590
:10583000801800F03FF810BD0122D207002800DBDD
:10584000101A002900DB511A8142704710B5202A36
:1058500004DB0146203A9140002010BD91402023F6
:105860009C1A0346E3401943904010BD10B5202A0E
:1058700004DB0846203AD040002110BD0B46D3403F
:10588000D0402024A21A91400843194610BD10B5FB
:10589000202A06DBCB170846203A1041C1170B43DC
:1058A00006E00B461341D0402024A21A9140084341
:1058B000194610BD002904DA401C490001D14008F6
:1058C0004000704770B40024050C05D1102400047A
:1058D00002D1002921D01124050E01D10002083483
:1058E000050F01D10001241D850F01D18000A41CEA
:1058F000002801DB4000641C002908D020252E1B55
:105900000D46F540A14000D001212943084301067E
:105910001B1B000ADB1D02D5002070BC7047DB0595
:10592000181880180029F8DA401C4900F5D170BC1D
:1059300040084000704710B5002B08DA0024401CD6
:10594000614192185B411A4301D14008400010BDEB
:10595000F0B51FB482B005460C0003D0084604F031
:1059600093FE02E004F090FE2030024600902146B3
:105970002846FFF76BFF049B059A04460F46184321
:105980001143084314D0184610431BD000984021FF
:105990000A1A18460599FFF769FF05460E46009A50
:1059A00005990498FFF752FF084305D0012004E051
:1059B0002046394607B0F0BD0020C11705430E430D
:1059C0002C43374300990E986305401A7905E40A81
:1059D00000220C43FD0A0A3002D500200146E9E707
:1059E0000105101969410C9C0D9D00196941FFF7D3
:1059F000A2FFDFE7FEB500231A461B1A8A4103DB2C
:105A00000020014603B0F0BD4A000D0301212D0B1B
:105A10000905520D0D43D10702D100186D41521EE8
:105A20005110FF31FF310131002704463E46384610
:105A3000009701910246012100200905FFF716FF9A
:105A4000C3197141F818324684468E464A41614670
:105A50002846611A904104D36046241A954176463F
:105A60001F46241900986D41401C00903428E1DD48
:105A7000F91930467041091BA84103D20022D243D4
:105A8000134601E00022134601980105381C7141BC
:105A9000FFF751FFB6E70000064C0125064E05E072
:105AA000E36807CC2B430C3C98471034B442F7D33F
:105AB000FFF70AFBC8C60008E8C6000870B58C18D6
:105AC0000578401C6B075B0F01D10378401C2A113D
:105AD00006D10278401C03E006780E70401C491C79
:105AE0005B1EF9D12B0705D40023521E0DD40B7079
:105AF000491CFAE70378401CCB1A921C03E01D787E
:105B00000D70491C5B1C521EF9D5A142D8D3002050
:105B100070BD000038B50446064805490068FFF727
:105B2000E7FA604300E0401E00900028FBD138BD3A
:105B300040420F0084010020F8B5044600688168E7
:105B40008907890F012902D10168C90722D181681B
:105B5000114A10261140012500290ED181682943E0
:105B600081600120FFF7D6FF01F030F807460CE016
:105B700001F02CF8C01B0A2807D9606D304360651E
:105B8000A06D2843A0650120F8BD20680068C043CF
:105B9000C007EDD10020F8BD170000801FB50B48ED
:105BA00000900B4801900B4802900B480390694607
:105BB0000A4805F05FF90A4A08481146083905F015
:105BC00047F800F077FA002004B010BDD5C40008F3
:105BD000B1C4000811C500080FC5000890010020DD
:105BE0001000002010B500231A4603E0845CE3187F
:105BF0009BB2521C8A42F9D3D84380B210BD000038
:105C000010B5034800F09EFD024800F09BFD10BD5A
:105C1000981700205017002030B5446C1C252C40EC
:105C20000125A540046C6560046863608368102BDF
:105C3000036803D099600068C26030BD9A60006854
:105C4000C16030BD1449012048720A4602205E320C
:105C5000507203203C3A507204200E3A50720F48A2
:105C60000D4B0078087022310870203108770C49FC
:105C70005A1C0878587149789971233318715971F1
:105C8000203318775977107551751A461E321075E2
:105C90005175107651767047E81100203E010020C2
:105CA0006001002010B503F025FE202003F0E0FE87
:105CB000012005F049FB002003F0DAFE044805F05E
:105CC000E7F9044805F096FC002005F0CBFC10BD78
:105CD0000001002083800000F8B5052001210007A5
:105CE00000F060FF0025174C002800D06560164EBC
:105CF0000221304600F056FF00281BD10120207001
:105D00001248808F00280ED00127BF02002239469A
:105D1000304600F054FF0A2004F00AFF0122394601
:105D2000304600F04CFF0A48656000880A2148436D
:105D300008490880012000F06DFE022000F06AFE94
:105D4000F8BD00007001002000040050E80D0020A4
:105D50004C0100205C0100207047000010B508498C
:105D600000224A6107494B684C1523434B604B683E
:105D7000082423434B60C009C001026010BD00002D
:105D8000E0170020002002407FB500250C460646A3
:105D9000039500F00FFEE009029003A9019600951B
:105DA000684600F09FFD002804D000F0D7FD0020D9
:105DB00004B070BD00F0D2FD0120F9E710B500235A
:105DC00002E0C45CCC545B1C9342FAD310BD0000CB
:105DD00010B5214A00219069C305204804D54169C6
:105DE000022319434161911593699B0505D54369C8
:105DF0000124234343616302194393695B0505D57D
:105E00004369082423434361E301194393691B0554
:105E100005D543690424234343616302194393690D
:105E20009B0405D54369102423434361630219434E
:105E300093699B0304D5446920231C43446119439F
:105E40009369DB0305D54369402423434361A002E2
:105E50000143916110BD000000200240E0170020C6
:105E600070B5054600F0B2FE0646184C0AE0681C04
:105E700008D0002D04D000F0A9FE801BA84201D953
:105E8000032070BDA069C007F1D1A069800701D5CA
:105E90000220A061A069C00511D4A06980050ED4BC
:105EA000A06940050BD4A069000508D4A06980044E
:105EB00005D4A069800302D4A069C00303D5FFF70D
:105EC00087FF012070BD002070BD0000002002404F
:105ED000F8B51746002605460C4600F06BFD09E0B4
:105EE00029460220226800F047FD002804D1241D25
:105EF0002D1D361DBE42F3D300F030FDBE4201D24F
:105F00000020F8BD0120F8BD10B508490246002068
:105F1000054B497905E044001C5B944203D0401CCA
:105F2000C0B28842F7D310BD8C130020700000204F
:105F300010B500F03CFE10BD10B5094801F028F87E
:105F400080B2FFF7BDFB074A074BFFF79DFA00221F
:105F5000064BFFF701FBFFF7F9FB80B210BD000015
:105F600004160020F853E3A59B843E4000408F4078
:105F700070B50024204603F03FF947494748A20086
:105F8000641CE4B28150142CF9D3464944480A7881
:105F900002754978417544490A7802764978417614
:105FA0003F490520133148720A2005F013FB7D207C
:105FB000400105F029FB3A49002213310C2005F07D
:105FC000F3FB00210C2005F001FC384800F0E0FF55
:105FD000344C0125223CA084AD0309E0334800F095
:105FE000D7FF80B2A084618EFF392D39884206DB4D
:105FF000618E80B28842F1D349198842EED80220DE
:1060000005F038FB002003F0F7F8294D00210F20A0
:1060100005F060FA2842E063F8D0E06B411C38D00C
:10602000400435D58122D20100210F2005F091FBDB
:106030000021102005F04EFA41061948490E0022B1
:10604000C73005F07DFA164DC735687A05281FD18F
:1060500002221549681DFFF7B5F8002818D111482C
:10606000AE7C66710422691C3230FFF787F829463E
:106070001331084672000D466930FFF77FF86079EA
:106080002946420005484838FFF778F80320207079
:1060900070BD04F06DFB0000FFFF0100EC13002059
:1060A0004912002092000020600100200416002008
:1060B00000D0272410B5144C144822461032114643
:1060C000083904F0C5FD0022114BE168A068FFF714
:1060D00043FA104A104B05F08DFC00220F4BFFF7DE
:1060E000CBF900220E4BFFF7CFF9FFF789FB2060B9
:1060F00000221346E168A068FFF75AFB01D0206830
:1061000010BD0020206010BD000000209001002084
:1061100000AA8F406C45D9CC955BC83F0000F03F8A
:1061200040A5E54010B5084800F096FA0A21064857
:1061300000F032FA044800F01DF9800503D502484A
:1061400000F01AF980B210BDA8150020F8B52F4D47
:1061500000220121284600F032FDFFF7E3FFFFF7A0
:1061600094FA2B4E3146FFF793F82A4C0122A06097
:106170001146284600F023FD2749A06800258842E3
:106180003EDB2078254F002815D02570FFF7CAFF89
:10619000FFF77BFA3146FFF77BF8A060FFF7F4FAD0
:1061A00000223B46FFF762F900221D4BFFF76CF916
:1061B000FFF726FB6060A068FFF7E6FA00223B4687
:1061C000FFF754F9174A184BFFF75EF906460F46DA
:1061D0006068FFF7D9FA134A144B5242FFF754F99B
:1061E00032463B46FFF79EF8FFF70AFB1049606016
:1061F000884201DD616004E0FF21C905C84200D387
:1062000065606068FFF76AFAC0B2F8BD000400502C
:1062100000401B44480000200000604000000C408B
:1062200000E064403333333333B33040CCCCEC3F05
:106230000000C842F8B5054604464035287C0026D3
:10624000012808D001202874206881688907890FF7
:1062500001290ED101E00220F8BD0168C90708D06C
:10626000606D2021084360650126002028743046B7
:10627000F8BD616DFF220132914302221143616535
:10628000C1688907890F0091C16889088900C160C8
:106290002068816892071143816000F097FC0746EF
:1062A0000EE000F093FCC01B0A2809D9606D0221A2
:1062B0008843102108436065002028740120F8BD40
:1062C000206880680028ECDB2068C168009A1143D0
:1062D000C160606D80088000401C6065C5E70000FB
:1062E000F8B506460D464036317C01290DD0012116
:1062F000317401688A68520709D5416D2022114323
:106300004165002030740120F8BD0220F8BD174B14
:106310006A68D80547109A42154C8A6A2B6812D0D1
:106320005B035B0B1A438A622968490305D5A168A0
:106330000143A1600A20FFF7EDFB2868800312D516
:10634000A06838430EE05B035B0B9A438A622968BE
:10635000490302D5A1688143A1602868800302D562
:10636000A068B843A06000203074F8BD01100000A0
:1063700000270140406D70470068006C70470000C6
:1063800070B5040006D0606D264600254036002812
:1063900002D006E0012070BDA5653574204600F0EE
:1063A000D3F8606DC00603D421688868400705D51E
:1063B000606D1021084360653574EBE7606DFF2266
:1063C0000132904302221043606588688207920F71
:1063D0005B48012A02D10A68D2072BD103236268E5
:1063E0009B079A4205D05B429A4202D05B009A42D8
:1063F00009D10A69920092080A6121680A696368F2
:106400001A430A610CE00A69920092080A618168E5
:106410000F22920491438160816862681143816018
:106420002168CA6818239A43CA602168CA68A368A9
:106430001A43CA60816801225206914381608168D3
:10644000A28E52061143816020688168C90004D47D
:10645000816801221207114381602068C168394AAE
:106460001140C1602069E168022825D00020014365
:10647000204620300278037B52035B001A4311430D
:10648000226B1143A26992031143E269D2031143C3
:106490002268D3681943D160616A0A46FF3AC23A5A
:1064A00005D0A26A11432268D3681943D1604278AB
:1064B0000121012A02D00BE00420D8E7007800284F
:1064C00023D0606D202210436065A06D0843A06555
:1064D000E06B012820681FD00169C90703D001695A
:1064E00049084900016120684169C908C900416142
:1064F00020684169A26B11434161A565606D800808
:106500008000401C6065002070BD2068C2680123C7
:106510001B041A43C260DBE70269FF239B009A4316
:10652000026120680269236CA66C1A43636C3343D2
:106530001A430261206802690A430261D3E700003E
:10654000002701401902FEFF10B586B00446142151
:106550006846FEF72CFE0E492068884216D10D4889
:10656000416B421511434163C16A01221143C1626B
:10657000C06A6946104005900220009003200190F7
:10658000002002900520000700F050FA06B010BD70
:106590000024014000100240F8B504464069254639
:1065A00040350E4608280BD02068C068C00709D0C7
:1065B000606D202108436065002028740120F8BD2B
:1065C000082700E00C2700F001FB009011E0701C90
:1065D0000FD0002E05D000F0F9FA0099401AB04211
:1065E00007D9606D042108436065002028740320EA
:1065F000F8BD206800683842E9D0606D0121490289
:10660000084360652068C16809058A0F0C21002ACB
:106610001BD12022125D002A17D10268120714D55F
:10662000826853070122002B08DB43688B434360D9
:10663000606D130298431043606506E0606D20238F
:1066400018436065A06D1043A065A069002801D1C2
:10665000206801600020F8BD70B504462168002064
:106660008968490721D425464035297C01291CD059
:1066700001212974E169012904D02046FFF75CFA61
:10668000002811D1616D0A4A1140FF2201321143E5
:1066900061650021A165297422681C2111602168AF
:1066A0008A6804231A438A6070BD022070BD00000E
:1066B000FEF1FFFF30B5014620314A790023022A5E
:1066C00004D00422C2630B71012030BD026814683B
:1066D0000E25AC43146002681468640864001460FA
:1066E000446C1C22144001221546006CA5404560F4
:1066F0004A7118460B7130BD70B500240146203137
:106700004A79022A03D00421C163012418E00268F7
:1067100013680E25AB431360026813685B085B00C7
:106720001360436C1C221340012215469D40036CEC
:106730005D604A7100220A71816B002900D0884790
:10674000204670BDF0B4016C0D6801680C68466CA1
:106750001C2304221E401746B7402F420ED0670765
:106760000CD50C68A40602D40C6894430C60416CF0
:1067700019408A40016C4A60016B1AE00227B74059
:1067800002462F402032002F17D0A70715D50C68DE
:10679000A40605D40C680A25AC430C600121517194
:1067A000446C02211C40036CA1405960002111710E
:1067B000C16A002918D0F0BC08470827B7402F420B
:1067C00012D0240710D50C680E25AC430C60446C25
:1067D00001211C400B46A340046C6360C1635171EE
:1067E00000211171416BE4E7F0BC704770B5040003
:1067F0003CD01F48256814212818FEF779FC80003A
:1068000060641C4820640221204620300246417109
:1068100029681948E3680140A0686669184323693C
:1068200033431843A3691843E3691843236A1843A1
:10683000084328600121A0688903884210D00D48D0
:106840008030836A656C1C210D400F26AE40B34337
:106850008362656C63680D40816AAB400B43836261
:106860000020E06301215171107170BD012070BDE5
:10687000F8FFFDBF000002400F80FFFFF8B504469F
:106880008C46203001790025012909D001260671A6
:1068900041790027012905D0077102252846F8BD56
:1068A0000220F8BD02214171E763206801684908B0
:1068B0004900016061462046FFF7AEF9206B0028D1
:1068C0002068016801D00E2205E004229143016096
:1068D000206801680A221143016020680168314381
:1068E0000160DBE7F8B51A4E0546307C0F460128FB
:1068F00007D0012030741748FFF7B2FA010002D028
:1069000021E00220F8BD0020C04338606C6814E02C
:106910002046FFF723FA0F48FFF7A2FA01460E4878
:10692000426808239A434260426843159A43426092
:10693000002901D03C6006E08034A8686A68C00184
:106940008018A042E4D8002030740846F8BD00004A
:10695000E017002050C300000020024005484168B5
:10696000022211434160416801221143416000202D
:106970007047000000200240F8B50C4C1646207C01
:106980000F46012808D0012020740948FFF768FA53
:106990000025002802D006E00220F8BD65613E60B7
:1069A0000348FFF75DFA2574F8BD0000E0170020EA
:1069B00050C3000011484168C9070BD0EFF31081A4
:1069C00072B60F4AC2600F4AC26081F310884168F4
:1069D000C9070ED1416889070DD5EFF3108172B652
:1069E000094A0261094A026181F310884068800700
:1069F00001D50120704700207047000000200240B0
:106A0000EFCDAB8905040302BFAE9D8C16151413A0
:106A10007047000010B504494A69024202D048613B
:106A2000FFF7F6FF10BD000000040140FCB5002395
:106A30000124A2E027462A469F403A406FD04D6885
:106A4000012D05D0022D03D0112D01D0122D16D10C
:106A500085680326AC465D00AE46AE406546B5434C
:106A6000AC46CE687546AE4065462E4386604668A5
:106A70000D79BE43ED06ED0F9D4035434560C66878
:106A80005F000325BD40AE46AE4335468E68BE402E
:106A90002E43C6604E68022E01D0122E14D1DE089D
:106AA000B60036180196366A5D07B446EE0E0F251D
:106AB000B54000966646AE43B4460D69009EB540AB
:106AC00066462E43019D2E6206687546AE430D79DB
:106AD000AD07AD0FBD40354305604D68ED004BD5AA
:106AE000294D6E6B26436E639E08284DB6007519BE
:106AF000AC46AD689E07360F0F27B740BD4305274C
:106B00003F07B84201D1002715E0214FB84201D11B
:106B1000012710E01F4FB84202D102270BE02BE003
:106B20001D4FB84201D1032705E01C4FB84201D1E7
:106B3000052700E00627B7402F436546AF60184D94
:106B40002E684F689643FF0300D516432E606E688B
:106B50004F689643BF0300D516436E60AE684F681A
:106B60009643FF0200D51643AE60EE684F68964329
:106B7000BF0200D51643EE605B1C0A681546DA407A
:106B800000D057E7FCBD00000010024000000140AB
:106B90000004005000080050000C0050001C005081
:106BA000000401400069084000D00120704742699C
:106BB00013460B401B0491430B4383617047002A2B
:106BC00001D0816170478162704700000148806890
:106BD0007047000078010020024881680278891817
:106BE000816070477801002010B5084800240168D2
:106BF000402211430160204600F00AF8002801D02D
:106C0000012401E000F00EFA204610BD00200240F1
:106C100070B504460D4D7D202978C000FEF768FA56
:106C200001460B480068FEF763FA00F095FE002865
:106C300009D1042C07D200222146401E00F00AFA96
:106C400000206C6070BD012070BD00007801002044
:106C50008401002070477047F8B502F017FF5A4CC6
:106C60000120E070208AFEF710FD01467F20C0055C
:106C7000FEF70EFB554D06462968FEF7B0FA286070
:106C80000120A16AC005814201DA084603E03046CE
:106C9000FEF7FAFAA062FF21C9050025C84200D319
:106CA000A562607800280BD102214948FFF77AFFDE
:106CB00002004849484818D00022FFF780FFE562EB
:106CC00002214348FFF76EFF444F454E002855D040
:106CD000E562B08AFEF7D9FC3C490968FEF7ACFDD5
:106CE0005FD24049012008705DE00122D1033A489B
:106CF000FFF765FF208AFEF7C8FC01467F20C0052C
:106D0000FEF7C6FAE16AFEF76AFA3749E06288429E
:106D1000D6DD33480127F926403000900A2130465D
:106D2000FEF7E6F9002903D12A492B48FFF700F9BD
:106D300002212748FFF736FF002801D0002701E095
:106D4000002F12D102212248FFF72CFF00280CD17E
:106D500004F018FE00990120888005F06FFB642084
:106D600003F0E6FE22492148C8600A2003F0E0FE55
:106D70003046761EF6B20028D0D1A1E7208AFEF771
:106D800084FC01467F20C005FEF782FAE16AFEF727
:106D900026FA1849E06288429BDB15491348C8600F
:106DA00097E710480570708F401EFEF763FC074997
:106DB0000968FEF741FD05D82079002802D001209E
:106DC0003870F8BD3D70F8BD3C0100207401002012
:106DD00000040050008000000000005083000020EC
:106DE000E80D002076000020000040400400FA0575
:106DF00000ED00E00000A04070477047704710B5FC
:106E0000044600680168C943C90708D18168C943BD
:106E1000C90704D1012141602046FFF71DFF20680A
:106E20000168C943890708D48168C943890704D424
:106E3000022141602046FFF70DFF20680168C94329
:106E4000490708D48168C943490704D40421416033
:106E5000204600F0E5F820680168C943090708D416
:106E60008168C943090704D4082141602046FFF71F
:106E7000C3FF20680168C943C90608D48168C943B3
:106E8000C90604D4102141602046FFF7E4FE2068C3
:106E90000168C943890608D48168C943890604D4B6
:106EA000202141602046FFF7A9FF20680168C943FF
:106EB000490608D48168C943490604D44021416089
:106EC0002046FFF79AFF10BDF8B5040005D025460F
:106ED0002035A87B002802D006E00120F8BD002064
:106EE0006873204600F03CF80220A8732068C2684E
:106EF00084466368012B01D10620824316486169EC
:106F0000814202D0072040038243002B01D1D820C8
:106F100082431248A668024018463043676A266AD0
:106F20003E433043A66A30431043002B02D0012B6E
:106F300004D005E02369E2691A4300E0E2681043E7
:106F4000054A914202D0A269114308436146C860D4
:106F50000120A8730020F8BDFFFF0000F8F119FF21
:106F600010B50068084988420CD10848816BC204FA
:106F700011438163002201210D2000F06BF80D20E8
:106F800000F05CF810BD0000007C004000100240E2
:106F90000068C06970470000F8B504460220254625
:106FA00020351746A8731D480268C3041A430260BF
:106FB0002068C2689B121A43C260206802690126D9
:106FC00032430261226810205060206881611021E4
:106FD000204601F0F9FB03281FD0216808204860F3
:106FE000206847610821204601F0EEFB032814D0F9
:106FF000204601F079FBA87B03280ED02068816829
:107000003143816020680169314301612068016971
:10701000042211430161AE730020F8BD0004014059
:10702000704700000448416B012211434163816BAA
:10703000020411438163704700100240002805DB01
:10704000C106C90E01208840014908607047000050
:1070500000E100E010B503F069FB10BD02480168D3
:10706000821511430160704700700040F8B5044676
:1070700000780027534D800671D5524E403EB06BCC
:10708000C00004D4B06BA9050843B06301274E4883
:107090000168C90511D40168821511430160FFF729
:1070A00095FD009005E0FFF791FD0099401A6428D6
:1070B00037D845480068C005F5D532680321090571
:1070C00060680A400140914208D08103890F03297A
:1070D00004D13168890301D50120F8BD2A69032153
:1070E00009040A4022D0084090421FD02078800630
:1070F0001CD528692A6988430121C9040A432A61E9
:107100002A698A432A612861C0050FD5FFF75EFD11
:10711000009008E0FFF75AFD0099411A2B48814280
:1071200001D90320F8BD28698005F3D5616888037B
:10713000800F032805D132680005824301400A43CD
:1071400032602869032261681204114008432861F3
:10715000002F04D0B16B012000078143B163207878
:10716000C00705D0E868A168800880000843E8608F
:107170002078800705D5E8680C218843E16808433A
:10718000E8602078400706D5E86803218902884333
:1071900021690843E8602078000706D5E8680321E4
:1071A0000903884361690843E8602078000606D532
:1071B000E868032189048843A1690843E860002046
:1071C000F8BD00004010024000700040881300002D
:1071D000F8B50E46050038D05E480068C007C00FFD
:1071E000B04214D25B4C206840084000304320601D
:1071F000FFF7ECFC074605E0FFF7E8FCC11B56482B
:1072000081427AD82068C007C00FB042F4D12878F4
:10721000524C800705D5E068F0218843A9680843EF
:10722000E0602878C00752D06868022806D003289A
:1072300007D0216801280AD0890504E02168890364
:1072400001E021688901002903DB0120F8BD49071D
:10725000F9E7E168890889000143E160FFF7B6FCBE
:107260000746686802280AD0032814D001281ED0D7
:1072700029E0FFF7ABFCC11B374881423DD8E068ED
:107280000007800F0228F4D121E0FFF79FFCC11B0B
:107290003148814231D8E0680007800F0328F4D1DB
:1072A00015E0FFF793FCC11B2B48814225D8E0680D
:1072B0000007800F0128F4D109E0FFF787FCC11B0C
:1072C0002548814219D8E0680007800FF5D1214890
:1072D0000168C907C90FB14217D9016849084900B7
:1072E00031430160FFF772FC074608E005E0FFF755
:1072F0006DFCC11B1848814201D90320F8BD154817
:107300000068C007C00FB042F1D12878400706D509
:10731000E068072109028843E9680843E0602878AB
:10732000000707D5E0680721C90288432969C90019
:107330000843E06000F03AF8E168094A0906090FDD
:10734000515CC8400749086007480068FFF760FCC7
:10735000F8BD000000200240881300000010024029
:1073600016C60008840100207C010020044805495D
:107370000068C968044A4905490F515CC840704714
:1073800084010020001002402FC60008044805496F
:107390000068C968044A8904490F515CC8407047B5
:1073A00084010020001002402FC6000870B51A4A60
:1073B000D3681A490C2018408D0004280CD04E00C8
:1073C000082810D00C2810D050680004410F01206C
:1073D000C003491C884070BD1068C00601D508462E
:1073E00070BD284670BD304670BD98020C4C000F31
:1073F000205C1B029C0FD368641CDB0301D5314663
:1074000003E01268D20600D4294603F054F922465C
:107410000023FDF783FE70BD0010024000093D000F
:1074200026C60008FEB505007ED0FE4CE7680C209D
:10743000E66807400120000406402878C00747D0CE
:10744000082F05D00C2F0AD101200004864206D156
:10745000206880033CD568680028E5D038E001202A
:1074600069680004814203D121680143216011E071
:10747000052301221B0492049942216802D1114381
:107480002160F1E78143216021680140009120687B
:1074900090432060686800280DD0FFF797FB0090AC
:1074A00005E0FFF793FB0099401A64287BD8206819
:1074B0008003F6D50CE0FFF789FB009005E0FFF7AD
:1074C00085FB0099401A6428F0D820688003F6D420
:1074D0002878800756D50923E868042F0DD00C2F93
:1074E00001D1002E09D000283CD0216899430143E6
:1074F0002160FFF76BFB064628E02168490701D5AC
:10750000002891D061681F22120291432A69120259
:10751000114361602168994301432160FFF746FFF1
:10752000E16809060A0F00E08BE1BF49895CC840A9
:10753000BE490860BE480068FFF76AFB002873D1A7
:1075400020E0FFF743FB801B0228AFD820684007EC
:10755000F7D560681F210902884329690902084399
:1075600060600FE02068400840002060FFF72EFBBD
:10757000064604E0FFF72AFB801B022896D8206805
:107580004007F7D42878C00660D5002F0CD0A86932
:1075900000284AD02068FF21013108432060FFF70E
:1075A00015FB06462EE0C1E02068800502D5A869DB
:1075B0000028A6D06068072149038843296A084348
:1075C00060606068297F0002000A09060843606065
:1075D000286A410B0120C003491C8840E168090664
:1075E0000A0F9149895CC84090490860904800683A
:1075F000FFF70EFB002817D128E0FFF7E7FA801B02
:107600000228A2D820688005F7D5606807214903C1
:107610008843296A084360606068297F0002000A85
:1076200009060843606011E0E2E02168FF200130B4
:1076300081432160FFF7CAFA064604E0FFF7C6FA65
:10764000801B022872D820688005F7D42878794EEC
:10765000000724D568690028306910D0012108434B
:107660003061FFF7B3FA009005E0FFF7AFFA009939
:10767000401A02285AD830698007F6D50FE0400832
:1076800040003061FFF7A2FA009005E0FFF79EFA94
:107690000099401A022849D830698007F6D4287822
:1076A000400766D500200290A06BC00006D4A06BF6
:1076B000012109070843A063012002905E48016888
:1076C000C90511D40168821511430160FFF77EFAE4
:1076D000009005E0FFF77AFA0099401A642825D84F
:1076E00055480068C005F5D5FF20AA6801308242E0
:1076F00003D131690143316111E001218902002A7E
:1077000007D005231B029A4203D132690A43326132
:10771000EFE7326982433261306988433061A8689B
:10772000002810D0FFF752FA009008E05FE0FFF762
:107730004DFA01460098091A4048814257D83069ED
:107740008005F4D50DE0FFF741FA009006E0FFF761
:107750003DFA0099411A3948814248D8306980057C
:10776000F5D40298002804D0A06B012109078843B2
:10777000A063686A002866D00C2F3ED0012636062A
:107780000228206805D0B0432060FFF71FFA0546A5
:107790002FE0B0432060FFF719FA074604E0FFF737
:1077A00015FAC01B022822D820688001F7D4E96AA4
:1077B000A86AE2680843296BFD231B049A4311431E
:1077C0000843E060206830432060FFF7FFF905467A
:1077D00004E0FFF7FBF9401B022808D8206880016D
:1077E000F7D530E0FFF7F2F9401B022801D903205A
:1077F000FEBD20688001F5D425E00128F8D0E068BE
:1078000001210904AA6A014091421AD10F21890479
:10781000EA6A0140914214D1032189050840296B8D
:1078200088420DE00010024016C6000884010020C6
:107830007C010020401002400070004088130000CE
:1078400001D00120FEBD0020FEBDF8B504000ED021
:10785000FF27606A0537002500280AD02561656189
:1078600026464036A562707C002807D00AE0012039
:10787000F8BD6068B842F3D0E561F1E735742046A1
:1078800000F03EF8022171742068026840239A4398
:1078900002602123A26860689B021A4038401043AE
:1078A000E3688A021340184323690B40217D184383
:1078B000C907C90F0843A169931019400843E1693A
:1078C000382319400843216A802319400843A16ADC
:1078D00093001940084321680860A0690421000C46
:1078E0000840616A102319400843216848602068F5
:1078F000C1699143C1616565012070740020F8BDC4
:1079000010B586B0044614216846FDF750FC1049B6
:107910002068884219D10F48416B8214114341639A
:10792000C16A01221143C162C06A00211040059062
:10793000E020009002200190032003900291049126
:10794000052069460007FFF771F806B010BD00007A
:107950000030014000100240094910B5401E884225
:1079600001D9012010BD074C60610321081F02F0FE
:10797000DDFE0020A06107202061002010BD000076
:10798000FFFFFF0000E000E0F0B502462032137E6A
:10799000012B1ED0012515760223537606687468E4
:1079A000B3687027BC430F68274377600068AC0753
:1079B000A04205D0084CA04202D0084CA04204D1FD
:1079C00080244968A34319438160557600201076CE
:1079D000F0BD0220F0BD000000080140001401408D
:1079E00070B5050005D02C462034607E002802D0FA
:1079F00006E0012070BD00202076284600F010F837
:107A000002206076291D286802F0B6F80120A077D0
:107A1000A076E076207760776076002070BD000069
:107A2000006801218907884204D10348816B012243
:107A3000114381637047000000100240F8B505460D
:107A400004462035287E012817D001262E760220F4
:107A50006876226890687727FF23B8431B02984313
:107A600090600A68502A31D00EDC202A4BD006DC08
:107A7000002A48D0102A3AD145E00220F8BD302A29
:107A800041D0402A33D136E0602A27D0702A12D064
:107A900001200003121A2AD0824228D1CB684A68FA
:107AA0008968206802F0A1F82068816801229203A9
:107AB000114381601BE0CB684A688968206802F046
:107AC00094F8216888683843886010E0CA6849687B
:107AD000206802F004F95021206806E0CA6849686D
:107AE000206802F00DF96021206802F089F86E76B6
:107AF00000202876F8BDCA684968206802F0EFF8CF
:107B000040212068F1E711462068EEE710B586B005
:107B1000044614216846FDF74AFB012120688907C5
:107B2000884212D10A49CA6A02200243CA62C96A5B
:107B300001900140059141020091002102910391C1
:107B4000049069460348FEF771FF06B010BD0000BF
:107B50000010024000040050F8B5064604462036E6
:107B6000307E0D4601280BD0012008273076002AF0
:107B700008D0042A16D0082A2AD00C2A4DD137E082
:107B80000220F8BD206802F043F82068816939437B
:107B90008161206881690422914381612068816943
:107BA000EA6812E0206802F04BF82068816901223F
:107BB000D2021143816120688269012189028A43CE
:107BC000826120688169EA6812021143816124E0C0
:107BD000206802F04EF82068C1693943C16120680D
:107BE000C16904229143C1612068C169EA6812E059
:107BF000206802F059F82068C1690122D2021143BD
:107C0000C1612068C269012189028A43C26120687A
:107C1000C169EA6812021143C16100203076F8BDE3
:107C200070B5050005D02C462034607E002802D0B7
:107C300006E0012070BD00202076284600F00FF8F5
:107C400002206076291D286801F096FF0120A077A8
:107C5000A076E076207760776076002070BD704770
:107C600070B505462C4602202034002908D004298E
:107C70000BD008290ED0627F012A10D0012070BDE0
:107C8000A27E012AFAD1A0760AE0E27E012AF5D18D
:107C9000E07605E0227F012AF0D1207700E06077CE
:107CA0000122286801F094FF01222868920701212F
:107CB000904205D0074A904202D0074A904204D130
:107CC00082685207520F062A02D002680A430260F5
:107CD000002070BD000801400014014070B504464A
:107CE0000D460068002201F073FF2068016A0C4A0B
:107CF000114203D101684908490001600120203484
:107D0000002D06D0042D06D0082D06D06077002067
:107D100070BDA076FBE7E076F9E72077F7E7000093
:107D2000111100007047704770470000F8B50268F5
:107D30000446D06911689668814B05461D40202392
:107D4000002D6CD0F7077F4DFF0FBC460D402F4331
:107D500079D02546C7078035002F06D0CF0504D53A
:107D6000012717622A683A432A60820708D5F2077A
:107D700006D0276802223A622A6804273A432A601A
:107D8000420708D5F20706D02668042232622A6824
:107D9000022632432A6002070AD50A461A4066467E
:107DA000324305D02668082232622E6816432E60C0
:107DB000020508D54A0106D501222668D2023262A0
:107DC0002A681A432A602A68002A30D0800606D51D
:107DD000880604D5616E002901D0204688472868AE
:107DE00021688968490602D42821084225D0204606
:107DF00002F0A7F920688168490619D582684021F8
:107E00008A438260206F002812D04F498163206F1F
:107E1000FEF772FC00280AD0206F816B06E0850611
:107E200011D58D060FD5616E77E020468847F8BDE5
:107E30002046FFF779FFF8BD05E02046FFF774FF05
:107E400000202860F7E7256E012D56D1C50654D5D0
:107E5000CD0652D51026166220688168254649064F
:107E6000403500292ADA226F116849680904090C93
:107E7000E1D02F8B8F42DED96983116809688906AA
:107E800017D4016832019143016020688168490874
:107E90004900816020688168402291438160E367E6
:107EA0000020206620680168B1430160206FFEF762
:107EB00001FC288B698B401A81B21AE0298B6A8BEE
:107EC000891A6A8B89B2002AB5D00029B3D002681A
:107ED000FF252135AA4302602068826852085200BB
:107EE0008260E36700202066606620680268B24313
:107EF00002602046FFF716FF9DE7C50208D5750210
:107F000006D50120000510622046FFF70CFF92E71E
:107F1000050605D50D0603D5A16E002985D18AE792
:107F2000400688D5480686D5116820464024A143DE
:107F3000116083670021816600F043F97BE7000050
:107F40000F0800002001000469A0000810B504001B
:107F500003D0A06F002802D007E0012010BD00214F
:107F600074200155204600F027F82420A0672068DF
:107F70000168490849000160204602F035F90128EE
:107F8000ECD0606A002802D0204601F04DFF206846
:107F900041680922D20291434160206881682A2207
:107FA00091438160206801680122114301602046ED
:107FB00001F0A0FF10BD0000F0B587B00646142107
:107FC0006846FDF7F4F82C493068884251D12B48B7
:107FD000416B0122920311434163C16A01221143A3
:107FE000C162C06A00251040059003204002009045
:107FF0000220032701A9A1C104200490052069469D
:108000000007FEF713FD1F4C1D48A560E56081C405
:108010008027E560A7602020256160610002A061E3
:108020001848083CFEF7E2FB002801D0FDF794FE5B
:108030003467A662144C124821461438206003208D
:10804000606010200831A1C16561A561E56120462D
:108050002562FEF7CBFB002801D0FDF77DFEF4661C
:10806000002201211B20A662FEF7F4FF1B20FEF771
:10807000E5FF07B0F0BD00000038014000100240ED
:1080800030000240501700209817002070B5C36FD1
:10809000202B27D100290BD0002A09D00124836886
:1080A0002403A34206D10369002B03D1CB0701D0DF
:1080B000012070BD034660331C7D012C12D00124C9
:1080C0001C7500230366084C0368A34207D05C6854
:1080D000240204D51C680125AD062C431C6002F067
:1080E00083F970BD022070BD0048004070477047A2
:1080F000FFB50446806F83B017460D4620285ED139
:10810000002D0AD0002F08D0A168C001814207D1FC
:108110002069002804D1E80702D0012007B0F0BD93
:10812000204660300090007D012848D00098012151
:1081300001750020802108512120A067FEF746FD2F
:10814000264640360190378277820120A1680003DD
:10815000814202D12069002805D02F4600250099D0
:108160000020087511E00027F9E700228021204651
:1081700002F080F9002815D1002F15D02168387839
:1081800088627F1C708A401E7082708A019B002862
:1081900006980090E9D100224021204602F06AF9B9
:1081A000002808D00320B9E728882168C005C00D41
:1081B0008862AD1CE6E72020A0670020AEE7022021
:1081C000ACE77047034D044C04A002F053FAE5609D
:1081D000FAE700000400FA0500ED00E0486172646F
:1081E0004661756C745F48616E646C65722E0D0A31
:1081F0000000000070B586B014216846FCF7D7FF78
:108200000F480124418B002900D14483408B012871
:1082100005D0022801D100F001FC06B070BD01229A
:10822000084E950229463046FEF7C9FC002102910E
:1082300003910095019469463046FEF7F7FBECE7A1
:108240003C0100200004005010B505242407002242
:1082500004212046FEF7B3FC002208212046FEF749
:10826000AEFC0A2002F06BFC012204212046FEF73E
:10827000A6FC0A2002F063FC002204212046FEF73F
:108280009EFC10BD10B505242407002204212046C1
:10829000FEF795FC012208212046FEF790FC0A20FB
:1082A00002F04DFC012204212046FEF788FC0A2042
:1082B00002F045FC002204212046FEF780FC10BDA0
:1082C000F8B5002405260746254636070022042176
:1082D0003046FEF774FC0A2002F031FC0122042132
:1082E0003046FEF76CFC6006040E08213046FEF7AF
:1082F00059FC002801D0641CE4B2052002F01FFCE8
:108300006D1CEDB2082DE1D3002F03D0FFF79CFFC9
:108310002046F8BDFFF7B6FFFAE770B5052605461B
:108320003607002204213046FEF749FC0024E80904
:1083300001D0012200E0002208213046FEF73FFC78
:108340006806050E0A2002F0FAFB012204213046DD
:10835000FEF735FC0A2002F0F2FB00220421304631
:10836000FEF72DFC0A2002F0EAFB641CE4B2082CA4
:10837000DDD370BD10B50524240701220821204655
:10838000FEF71DFC012204212046FEF718FC002206
:1083900008212046FEF713FC0A2002F0D0FB002241
:1083A00004212046FEF70BFC10BD10B50524240760
:1083B000002204212046FEF702FC0022082120466C
:1083C000FEF7FDFB0A2002F0BAFB01220421204641
:1083D000FEF7F5FB012208212046FEF7F0FB0A20FC
:1083E00002F0ADFB10BD70B505252D07002401225C
:1083F00008212846FEF7E3FB062002F0A0FB01223D
:1084000004212846FEF7DBFB062002F098FB07E07C
:10841000641CE4B2FA2C03D9FFF7C7FF012070BD3A
:1084200008212846FEF7BEFB0028F1D100220421D6
:108430002846FEF7C4FB002070BD0000F8B501F02F
:108440008BFD01F0C5FD5B480068C069FDF774FD58
:10845000594C5A49A082898F594E0025002931D0A4
:10846000A26A730357499A4202DB02220A7000E0B3
:108470000D700A7801218902002A05D0012A0ED048
:10848000022A10D0032A1DD1608B01282ED0022889
:1084900018D1484808214038FFF720FC12E0FF229D
:1084A000F5329042F0D2608B01281DD0022804D012
:1084B00008E03046FEF783FB04E03E4808214038E0
:1084C000FFF7CEFBFDF742FE20700121C9023046C6
:1084D000FEF768FB0127FF0300282DD03A4805600E
:1084E000A079002804D007E00022E2E70122E0E7BB
:1084F0000120A07102F020F880213046FEF752FBE7
:10850000002806D0002208213046FEF758FB012241
:1085100005E0012208213046FEF751FB002205202C
:1085200039460007FEF74BFB244C284E4034A08C04
:10853000274F012803D01CE0A5710022EAE7254857
:108540006946088072B680212348FDF71DFC00288B
:1085500004D0022269462048FDF7BAFC62B61FA08B
:1085600002F088F8A58403F069FF642002F0E0FAC5
:10857000FE60608C012808D110486584058003F0F6
:108580005DFF642002F0D4FAFE60208C012806D141
:10859000258403F053FF642002F0CAFAFE60074806
:1085A000124A0188914202D1C088002800D1FE60A1
:1085B000F8BD0000CC1600203C010020E80D002092
:1085C0000004005081000020740100200400FA051E
:1085D00000ED00E0AAAA0000384A0008BDF8C8EB88
:1085E000C9FDBCB6C4A3CABD0D0A0000AA5500004F
:1085F00008B55721202000F06AF80321212000F05F
:1086000066F84021222000F062F80821232000F0C3
:108610005EF8AA21302000F05AF8084801210187AD
:10862000322000F054F80221332000F050F8684660
:1086300000F006F80A2002F082FA08BDE80D0020DA
:1086400010B501460F2000F021F8002800D00120CD
:1086500010BD10B50446FFF78DFE3220FFF75DFE1A
:10866000FFF7C1FEE0B2FFF758FEFFF7BCFEFFF7D1
:1086700081FE3320FFF751FEFFF7B5FE0020FFF724
:108680001FFE0446FFF791FE204610BD10B50C46B4
:10869000FFF7DFFF2070012010BD70B50D460446C6
:1086A000FFF768FE3220FFF738FEFFF79CFEE0B2CE
:1086B000FFF733FEFFF797FE2846FFF72EFEFFF782
:1086C00092FEFFF772FE0A2002F039FA70BD10B573
:1086D000FFF7E3FF012010BD10B50248FEF78FFB46
:1086E00010BD000004160020FEB50446002772B637
:1086F000334A01688B1804D13248C76803208004CC
:10870000074088680190C868009048698E69002B0E
:1087100008D12C4940398B6ACD042B438B628B6A7C
:10872000AB438B62014631433CD025492368CB42A1
:1087300005D12449CA6803239B049A43CA6025468D
:108740002035002810D021680A6901231A430A61E4
:10875000216848610821204600F036F8032800D13E
:10876000A873216808204860002E10D02068016995
:10877000012211430161206886611021204600F02A
:1087800023F8032800D1A8732168102048600C4802
:108790002168C14206D10B48C1680322920491436B
:1087A0003943C160206801694908490001612168B5
:1087B0000198886021680098C86062B6FEBD00001C
:1087C0000084FFBF4010024070B506460B480D46BE
:1087D000002409490068FCF78BFC7D21C90048434F
:1087E0003168401E00D103240B682A469A4301D009
:1087F0000028F6D1204670BD204E000084010020E4
:108800001CB5002116480091144A01910260C16311
:1088100012054260816007228263012202610246E2
:10882000C16020321170FF235170C23343628162F4
:10883000117301638161042241634261C161FDF7EB
:108840009FFD084800908013019069460448FDF799
:1088500047FD00210248FDF7EDFC1CBD002401404E
:10886000A81500200200000408B50848016B012289
:1088700011430163006B01211040009000220A2087
:10888000FEF7E8FB0A20FEF7D9FB08BD0010024006
:10889000F0B587B014216846FCF789FC4748C26AE6
:1088A00004210A43C262C26A0A400592C16A802654
:1088B0003143C162C16A31400591C16A012421433B
:1088C000C162C16A21400591C16A02252943C16282
:1088D000C06A22462840059005201C210007FEF7AB
:1088E0006EF9012236493748FEF769F90022364908
:1088F0003448FEF764F9912105200022090200079F
:10890000FEF75DF93148019000270520694602977E
:1089100000940007FEF78AF80C20009011200190C7
:10892000032003900520029769460007FEF77EF8B2
:1089300010206A46039591C2052069460007FEF79C
:1089400075F81120019002976946039700941D481D
:10895000FEF76CF81E48019069460095029419488C
:10896000FEF764F8E0020090694601970295154809
:10897000FEF75CF81748694691C1694611480397AC
:10898000FEF754F891200002694691C1052069461E
:1089900000070397FEF74AF869460A4801970096D0
:1089A0000294FEF743F8002201210520FEF752FB56
:1089B0000520FEF743FB07B0F0BD000000100240A9
:1089C00001020000000400500830000000001110F7
:1089D000000021100832000010B50F4C0D48206037
:1089E000FF20053060600020A060E06020616061D1
:1089F000E0610121206249026062A161A06207205A
:108A0000E0622046FEF721FF206801684022114302
:108A1000016010BD003001403416002010B58AB04E
:108A2000002404940594069407940894012118489E
:108A30000994009401940294890703940160092128
:108A400084604160046113494461C160FEF7C8FF5E
:108A500001200003049004A90D48FEF7EFFF0C4825
:108A6000FFF7DEF8089408A909480994FEF78CFF7F
:108A700060200090084801900294082269460394FF
:108A80000348FFF769F80248FFF740F80AB010BD45
:108A90008C160020930400005702000000B585B03A
:108AA00014216846FCF783FB0E480D490160E12163
:108AB0004902416000218160C160016181610C2235
:108AC000C161426101623021416201210903816378
:108AD0004900C163FFF73AFA01F028FD05B000BD77
:108AE00000380140CC16002070470000F0B589B076
:108AF0000A2002F06FFD7D20400102F085FDFB4C55
:108B00000025A570FA48E065A07B0C2801D30B2056
:108B1000A07360790A2801D90A206071F548E570D0
:108B2000F54E00783071F549A07909784000084386
:108B3000E17C89000843F071A06BF070010A31728A
:108B4000401CA0636079B07442003046EC49133099
:108B5000FCF714FB6079EA4982004000801960311B
:108B60001330121DFCF70AFB6079062142004843CE
:108B70008019E4491730921CFCF700FB2A20205E84
:108B8000002803D0E049098A081860856079D74930
:108B9000C000223182190B7A53764B7A93760622E3
:108BA0007272DA4A1D301278B272228C3273D24A53
:108BB0000B78133A1375497851750022CE4902F0AB
:108BC000F3FD60790021C0001D3002F0FFFDD048A8
:108BD000FEF7DEF90127A084BF0309E0CC48FEF7C9
:108BE000D7F980B2A084618EFF392D39884206DB27
:108BF000618E80B28842F1D3C9198842EED8022032
:108C000002F038FD01221103C248FDF7D8FFBA482F
:108C10000126C571E573E57266732573BC48FEF7DE
:108C2000B7F9E0840746E5706079FCF749FDBA4A78
:108C3000BA4BFCF729FC01F017FF0022B84BFCF7F8
:108C400071FBFCF783FD0006C10CC81980B2F1036B
:108C50002085884201D3401A2085B248A06420793B
:108C6000401C2071AA48FEF793F9A084A4489F4FA6
:108C7000643840370690B5E1A548FEF789F9A0842D
:108C80000BE0A348FEF784F980B2A084218D8842CE
:108C900003D3A54A8918884207D300210F2002F088
:108CA00019FCA249E0630842EBD0E06B411C20D0E4
:108CB00040047DD58122D20100210F2002F049FD20
:108CC0007D20400102F0A0FC002002F052FC0021B7
:108CD000102002F0FFFB41068948490E00227C3833
:108CE000A16502F02DFC86487C38417A0729C2D163
:108CF00001E001F03DFD02228D49401DFCF762FAC2
:108D00000028B8D102F0B3FDE167A06702F09CFD36
:108D1000764B803303C3E0787949401CE070833997
:108D20000B7A68460370497A417000880390618C21
:108D300088427DD170497F488C31C98E01806E494F
:108D40006A488C31098FC1837148FEF721F9A084EC
:108D500002F0D2FA6548FF22803001684068520470
:108D60000023891858410206080A104341084900A7
:108D700000900A0E08025D498031CA6088605E4832
:108D8000E36F0A30A26F02F047FD607981005A4814
:108D900008185649163080310CC902F03DFD534881
:108DA0008030C36882685448123002F035FD00E01C
:108DB0000BE1514808214172A07C002814D0504892
:108DC00002225B497738FCF7FDF900280CD14A48AC
:108DD000E673C671A06D4A491638C2B26639C81D1D
:108DE0002274FB30FCF7CAF9607900228000424906
:108DF0001C3002F0D9FC6079002180001C3002F0A8
:108E0000E5FC009802F0DFFB012002F033FC607209
:108E100002214048FDF7C6FE00281ED00021374839
:108E2000017035498C31488E0490B880888E00E0FE
:108E300084E00890F880606CFF310531A064086020
:108E4000DC39E064C97C8C460907090F032900D08E
:108E50006174A16D1C2902D015E00121DFE72649CC
:108E6000224A8C31C98F9185069B264A1B88138024
:108E7000884207DD002805DD002903D0607D401C05
:108E8000607500E0657560460009A0742571E672A2
:108E900004983881089878812673E08B2649FF3042
:108EA000C33080B2E08388420CD949424018E08345
:108EB00020487D220188D200491C89B2018091425C
:108EC00000D305801B487D210088C9004843E18B01
:108ED0004018206500F076FD607A002805D1002159
:108EE0000F2002F0F7FA0006F9D584E070000020A8
:108EF0003F420F003C0100205C1200207001002066
:108F00008C130020C8140020280E00204C010020E3
:108F10000416002000040050B81E85EB51B8CE3F67
:108F200000000840A0860100983A000000D02724E5
:108F3000600100206C010020E7030000FCF7E4FF63
:108F40006A4A032111546A494A8EBA80898EF9808F
:108F5000A26D1C2A06D1654B4200AC33D318069A89
:108F600012885A808000614A614B603A02905F49E2
:108F700082189B8F138030394118626C4A605C49BB
:108F80008C3940185B4916300CC902F045FCE16D84
:108F9000606C884208DA554A0299603A51580129B2
:108FA00002D1E065039905915049029A60398A58C7
:108FB000824217DD012A15DD2146002812DD0398C3
:108FC000488402200870A5720CE04B4A00210F2053
:108FD00002F0BFFB6079E178401C814202D00020A2
:108FE00002F0C7FAA18C208D814200D244E6434AA8
:108FF00080188142FAD8E07A012801D00220E0727C
:1090000002F07AF93C4A00210F2002F0A2FB012174
:10901000002209033A48FDF7D2FD2079002814D038
:10902000384909888A008A18824200D225700020B7
:1090300000F0E2F8E07B002836D02C490C310B78A8
:1090400048788A78022B17D02EE0A16CE26D323975
:1090500020468A420EDAC1792A4A491CC9B2C17136
:10906000128852008A42E5D205994184022101709A
:10907000A572DFE7E571DDE710280CD0C82813D210
:10908000214BC91C1818FCF779F803F0D7F96420B4
:1090900001F04EFD2DE61D4D28684000000E03D165
:1090A000C878FCF7F2FA286000202378A27A657964
:1090B0000FE00E4E4100903E775A1836765AB7426E
:1090C00005D00B4F0223002201268C377E52401C14
:1090D000C0B2A842EDD32370A272074A00218032A9
:1090E0000F2002F036FB09B0F0BD00001C14002078
:1090F000E8120020F000002000D02724983A000059
:10910000000400504C010020E80D00206401002004
:10911000F8B52E4C0546A06E2D4A281A411EE06671
:10912000914215D2EB218900081AFCF7B5FA294AB9
:10913000294BFCF7A9F906462E200F46205EFCF7C6
:10914000ABFA32463B46FCF7EDF8FCF7DBFAE0857C
:109150000020A0751D481823C35E028C1F4800889C
:1091600084461F4806881DE06046484380181D4F0E
:1091700080B23880302778436427643078431A4FB0
:109180002066C01985420BD2C8B218492E22088029
:10919000206EA25E411BC91889186166A066F8BDE1
:1091A000491CA175A17DB142DED330204243104855
:1091B0006421101848430F494118A16620662E21EA
:1091C000401B615EC01840186066F8BD700000204A
:1091D000CF0700009A9999999999B93F5A010020AF
:1091E0004C0100206E01002078ECFFFF58010020A8
:1091F00074270000C0BDF0FFF1B5284882B0018897
:10920000491C8FB207802648068826483146FBF75E
:109210006FFF254CA18E4518B74205D31F4800218A
:1092200001802248281811E00298FCF749FA204AE8
:10923000204BFCF729F906460F462846FCF740FA72
:1092400032463B46FCF76EF8FCF780FA2086012593
:1092500080B2ED03A84201D3401B2086608BFCF74F
:109260002FFA154A154BFCF777F90746208E0E4664
:109270000090FCF725FA3A463346FCF753F8FCF722
:1092800065FA80B26086A84201D3401B60860C4913
:109290000098096848610098A086FEBD580100202A
:1092A0004C010020E17A000070000020240500003D
:1092B0001904560E2D624040F853E3A59B843E40AE
:1092C0000416002070470000F0B589B0002004901B
:1092D0000A2002F07FF97D20400102F095F9B348A1
:1092E00000218170826BB34C521C8263B04A438D63
:1092F000128A2546D21842850175214613310791FD
:10930000223047310290313520461338AA4F03915D
:109310000590A64E0F21A948717100782071A84AC6
:10932000B079127840001043F27C92001043E07153
:10933000308FE070000A2072A17431461E229C31E9
:109340000798FBF71BFF402228469E49FBF716FFB4
:10935000029903980A7AC274497A017509206072E9
:1093600099480078A072308C2073307D41003046DF
:109370009C30091805980A7802754978417576205D
:1093800000228C4902F010FA70790621484300212E
:109390001C3002F01BFA022002F06CF900210F20B1
:1093A00002F098F83842F063F8D0F06B411C18D006
:1093B00040047DD58122D20100210F2002F0C9F99D
:1093C0000021102002F086F841067A48490E00225A
:1093D000B43002F0B5F87748B430417A022902D0AF
:1093E000BDE001F0C5F902227849401DFBF7EAFE15
:1093F0000028F5D16D480222007D41006B489C3069
:1094000009186C48B530FBF7DDFE0028E8D102F002
:109410002EFA664AD167906702F016FA634A8032E4
:1094200003C2049800282CD1012004906148684EA2
:109430008C30C08E5F4930805C488C31098FC1838D
:109440006448FDF7A5FD5949634A8884C88BFF30FD
:10945000C33080B2C88390420CD952428018C8836E
:1094600030885D4A401C80B20B323080904201D37C
:109470000020308030887D22D2005043CA8B801873
:1094800008654C4869468C30428E0A80808E488040
:1094900048490422B531C81FFF38FBF76FFE434827
:1094A000484A007D0099800011504049803100E019
:1094B00076E003C9FF235B040022C018514109066E
:1094C000060A0E43304602F07EF8710849000A0E83
:1094D0000802364900268031CA6088603348C36F6D
:1094E000826F3448483802F097F9304880300CC811
:1094F0003048443802F090F92C488030C3688268C4
:109500002C48403802F088F92A49002252393C2080
:1095100002F04AF900213C2002F058F9012002F043
:10952000A9F82249487208468078401C88700121B9
:109530000520C9030007FCF7FBFC1C48407A002803
:1095400005D100210F2001F0C5FF0006F9D58022CA
:1095500000210F2002F0FDF81448467002E0134984
:10956000012048701148017D491CC9B201750F29BD
:1095700000D2CEE60498002810D10C481749028C7E
:10958000002A02D00B889A4201D909880184144923
:10959000008C0988401E48431249088009B0F0BD7C
:1095A000114A00210F2002F0D4F8D8E77000002003
:1095B000280E00205C12002000D027243C0100204F
:1095C00070010020781400204C0100206001002070
:1095D0006C01002004160020E70300004801002071
:1095E000460100204401002000902724F8B53349AB
:1095F0003148086002F0C6F9314800F0A3F9314C57
:10960000E0822F48801C00F09DF920832C48001D2B
:1096100000F098F9608345212B48C9004180322130
:10962000C180014640310979284F0906090E617051
:1096300006D1C7800121C1870A2141870021818786
:10964000234AC18E1170C18F2171818F6171817A1E
:10965000A1708588052165626181C6883046FBF767
:1096600047FDA08101462846FBF742FD8800081807
:1096700085B2164825816843FCF722F8154A164B37
:10968000FBF76AFFFCF762F8E081658231463846F5
:10969000FBF72EFD20820146C820FBF729FDE08361
:1096A0000120A083FCF748FCA082E2890B490C480A
:1096B000FDF772FCF8BD000065A5000868000020F9
:1096C000004F00083C010020E80D0020E8030000E6
:1096D00018000020F853E3A59B843E40FF7F000064
:1096E00004160020F8B5744C00202071734D012041
:1096F0002880734EC8203080207A401C2072C0071A
:1097000006D0208C411E2184022801D2C82020844A
:109710000120FFF771FD0A2001F05CFF7D20400170
:1097200001F072FF02216748FDF73CFA00283FD0A4
:109730000020654980000978654F49000843634966
:1097400009780843B872102078726248C1887D2079
:10975000C000FBF7CDFC78735F485E490078B873B2
:1097600038460B308A780270C97841705949421CDA
:1097700020310B7ED370497E11715649D01C2231A5
:109780000B7E5371497E9171524940310A7C0271BE
:10979000497C417100223946172002F005F800216A
:1097A000172002F013F8022001F064FF4B4F03E092
:1097B0000120BEE7FEF742FE00210F2001F08AFEE5
:1097C0003842E063F6D0E06B411C73D040046FD5A3
:1097D0008122D20100210F2001F0BBFF00211020C7
:1097E00001F078FE41063A48490E0022B430A165E6
:1097F00001F0A6FE364FB437787A112858D10222EC
:109800003749781DFBF7DEFC002851D1F81F027A9A
:1098100069460A70407A4870B97A2980C820FBF7F7
:1098200067FC3080387B208438462E4D2838C08E27
:109830002880394620482839098FC1832A48FDF7F6
:10984000A7FBA084E08B2949FF30C33080B2E083BE
:1098500088420CD949424018E08328882349401C9B
:1098600080B20B312880884201D3002028802888CC
:109870007D21C9004843E18B4018206500F0A2F823
:109880006846008860841249B87CC7316071420024
:1098900008460D466930FBF771FC607929464200A5
:1098A0001348FBF76BFC208CFF2801D003202070AD
:1098B000F8BDFFE700F05CFF700000204C010020C5
:1098C0005A01002000040050400100204101002006
:1098D0005C120020E80D00201800002000D0272492
:1098E000600100206C01002004160020E703000046
:1098F000A413002070B586B014216846FBF757FC0E
:1099000001250F4EED03002229463046FDF757F999
:10991000012000240190029469460095039430468A
:10992000FDF784F8032001900294694600950394A2
:109930003046FDF77BF8022001F0FAF806B070BD62
:10994000000400500088704770470000F8B50446D6
:1099500000206A461080194D55222A70AA226A708A
:109960000322AA70661DEE702A716971144A4900BB
:109970008918AC712246E81DFBF700FC002007E0C7
:1099800029186A468978128889186A461180401C0D
:10999000B042F5DB611DA81CFCF724F901466846BE
:1099A000018029190078C8716846407808722146FC
:1099B0000931024800F0E6FBF8BD00004215002026
:1099C000E80D0020FEB5FFF7A3FB2548FDF7E0FA00
:1099D000244C86B2A68460790A21081AC000FBF7DD
:1099E0005BFE07460191606EFBF76AFE1E4A1F4B45
:1099F000FBF7B2FD00900D463046FBF761FE2B46AB
:109A0000009AFBF78FFC3A46019BFBF78BFCFBF7B8
:109A10009DFE85B22586608BFBF752FE124A134BE2
:109A2000FBF79AFD06460F462846FBF749FE3246ED
:109A30003B46FBF777FCFBF789FE81B20120C003B0
:109A40006186814201D3091A6186854201D3281AB1
:109A500020860349208E09684861A086FEBD00006B
:109A60000416002070000020F853E3A59B843E40BC
:109A7000034A1168382389B2994301431160704742
:109A80000030014010B5FDF7A7F810BD10B59AB031
:109A900034216846FBF78BFB14210DA8FBF787FBED
:109AA0001C2112A8FBF783FB1B4801680324E40276
:109AB000A143C21489180160FDF7D0FA1748016963
:109AC000A143016106200090FF2001300290012097
:109AD0000390102004900220099040040B90000194
:109AE00000240C900A946846FDF79CFC0F200D9012
:109AF00003200E900F941094012111940DA8FDF7EE
:109B000067FB81201290032080041890149412A8FF
:109B1000FDF7ACFA1AB010BD0070004040100240D2
:109B200010480168821511430160C1680E4A114056
:109B3000C16001680D4A114001608168490849000F
:109B4000816001680122920491430160C168FD2295
:109B500012049143C16000210161064904488860F4
:109B600070470000001002400C40FF88F6FFF6FE30
:109B70000050000800ED00E070B5026801239B076B
:109B8000114C124D984203D0A04201D0A84203D1FB
:109B90007026B2434E683243984203D0A04201D0AF
:109BA000A84204D103231B029A43CB681A438023A3
:109BB0009A430B691A4302608A68C262096881622B
:109BC0000121416170BD0000000801400014014006
:109BD00010B5CB06DB0E0121046A99408C43046268
:109BE000016A9A401143016210BD30B58468FF25B7
:109BF0002D021B021343AC430B432343836030BD50
:109C0000826870239A430A4307210A43826070479F
:109C100030B5026A520852000262026A45688369DE
:109C20007024A3439C080B68A40023430224A2438E
:109C30008C6845601443836149684163046230BDA8
:109C400030B5026A10239A430262036A456882694A
:109C500073242402A2430C68240214432022934359
:109C60008A68456012011A4384614968816302620F
:109C700030BD30B5026AFF2301339A430262026AA3
:109C80004568C3697024A3439C080B68A400234360
:109C900001246402A2438C68456024021443C3611A
:109CA0004968C163046230BD30B5026A01231B03F9
:109CB0009A430262036A4568C26973242402A2437C
:109CC0000C68240214430122520393438A684560BE
:109CD00012031A43C46149680164026230BD30B5A1
:109CE000036A046A6408640004628469F025AC4372
:109CF000120122430A24A3430B438261036230BD55
:109D000030B5036A1024A34303628469036A0F25F4
:109D10002D031203AC432243A024A343090119439A
:109D20008261016230BD0000F8B5102405252D07C1
:109D3000AC62AF20800000F002FFAC6101F0DEFBFE
:109D40002F4C304F304E20670EE001F0D7FB2067DC
:109D5000FEF774FB206C411C2164142804D92BA04D
:109D600000F088FC2D48C760206FB042EDD100267E
:109D7000266420780127FF03030000F0B4FC0504EB
:109D80000C192D303200012239462846FCF717FF06
:109D9000FFF7A8FC06E0012239462846FCF70FFF32
:109DA000FFF792FA002239462846FCF708FF18E030
:109DB000A07A0122401CA07239462846FCF7FFFE1B
:109DC000FCF7D6F8002239462846FCF7F8FEA07AC0
:109DD000052806D9267004E0FEF788FE01E0FFF7AB
:109DE00073FA02210E48FCF7DDFE002805D00020A2
:109DF0000C49087001F068FAF8BD0120F8E700008E
:109E0000700000200400FA053001CADE44572049E2
:109E100044204552524F522E0D0A000000ED00E042
:109E2000000400507001002010B5818CC90707D0D4
:109E300001684A6801235B049A43836A1A434A60B3
:109E4000818C890707D501684A6801231B049A435E
:109E5000C36A1A434A60818C490707D501684A687A
:109E600001239B049A43036B1A434A60818C0907C0
:109E700007D501684A680123DB039A43436B1A4301
:109E80004A60818CC90607D50268916801231B03CB
:109E90009943836B19439160818C890607D50168CA
:109EA0008A6801235B039A43C36B1A438A60818CDF
:109EB000490612D503685A6801210905046C8A43D2
:109EC00022435A60026C8A4207D102685168032318
:109ED0005B059943436C19435160818C090607D592
:109EE00001684A680123DB04806C9A4302434A609C
:109EF00010BD0000F8B50446002680300660FCF76F
:109F000065FE054620680068124F000709D501214B
:109F10002B46002249052046009700F0ABFA0028A6
:109F20000DD12068006840070BD501212B46002287
:109F300089052046009700F09DFA002801D00320F3
:109F4000F8BD2020A067E0672666603426750020F3
:109F5000F8BD0000FFFFFF01F8B5184CC826E078F7
:109F6000002829D16079002826D101206071144D84
:109F7000686B002700281ED0686BC821081A15E0FE
:109F80001048E168405C616988470F480A210088F1
:109F900048430E490880E068401CE060E068C8283B
:109FA00000DBE760696BC820401A761EE1688142D9
:109FB00001D0002EE4DC6771F8BD000054000020E1
:109FC00000000240200D00204C0100205C01002018
:109FD00070B5224CE07800283FD1207900283CD190
:109FE000012020711E4EF16900250906002933DA8F
:109FF0002156625791420AD1F06940062CD5A079CA
:10A00000002829D0A5712089401C208124E0A17955
:10A01000002903D1A0710A2000F091FD00202056F4
:10A02000CC2148430F494218206912181279B262B4
:10A03000401C00222061A256CC235A4389588142F9
:10A040000ADC25612078401C207020780E2800D181
:10A050002570A078401CA070257170BD54000020B0
:10A0600000380140F801002010B5806A0022014646
:10A0700040314A834A82FDF757FE10BD70B5846AAD
:10A08000A06FE56F2168896800260906002906DAB5
:10A09000212804D152200653204600F06BF8206896
:10A0A0008068400606D5222D04D15A20065320464A
:10A0B00000F047F82046803001681022114301600B
:10A0C0002046FDF731FE70BD10B501460968806A73
:10A0D000096889061CD400225A210A5201680A68BC
:10A0E000FF2301339A430A6001688A6852085200CC
:10A0F0008A6001688A6840239A438A602021C16788
:10A10000016E012904D101680A6810239A430A608C
:10A11000016E012902D0FDF7E9FF10BD5821095A4F
:10A12000FDF700FE10BD10B5806A016E012902D056
:10A13000FDF7DDFF10BD5821095A4908FDF7F2FD72
:10A1400010BD01680A68FF2321339A430A60016841
:10A150008A68520852008A60016E012904D10168A0
:10A160000A6810239A430A602021C1670021016612
:10A170004166704701680A68C0239A430A6020213B
:10A180008167704770B5164CE278002A0CD12279AD
:10A19000002A09D10122E2700025C82903DC02222D
:10A1A000A256002A01DCE57070BD0123E356CC22E3
:10A1B00053430C4AD1500123E356CC2673439B18DA
:10A1C0000A460146181DFAF7D9FF6078401C6070F6
:10A1D00060780E2800D16570A078401EA070E2E77C
:10A1E00054000020F8010020F8B50446016880689A
:10A1F0002369E66918436369002533431843724AAB
:10A200000B68724E334003430B6021684868032398
:10A210001B039843E368184348602168A069914292
:10A2200001D0236A18438B680B263602B3430343DD
:10A230008B606749236867488B420CD1C0688007F0
:10A24000800F06D0012839D0022835D0032821D12B
:10A250001EE001271FE060498B420AD1C0680C2133
:10A26000084027D0042829D0082825D00C2811D14F
:10A270000EE093420ED1C16803208002014019D044
:10A2800001208002091A19D0091A15D0814201D182
:10A29000082700E010274F49504840398600934274
:10A2A00032D1002F0CD0022F0DD0042F10D0082F48
:10A2B0007FD126E00027EEE70227ECE70427EAE754
:10A2C000FDF754F806E00968C90605D4304603E0F6
:10A2D000FDF76CF8002872D0626851005118814275
:10A2E00067D81103814264D3010E0602500800238F
:10A2F00030185941FAF712FF03210902411A384A6E
:10A3000055E00120C003E7E70122E369D20393424D
:10A310002BD13B0000F0E7F90906090C4D114D4D1A
:10A320004D274D00FDF722F809E0FDF72FF806E074
:10A330000968C90605D4304603E0FDF737F8002860
:10A340003DD0616840004A088018FAF7D1FE80B21B
:10A350000146244A103991422BD8511C0140000774
:10A36000400F084329E01046EBE73B0000F0BBF943
:10A370000906090C2112212121232100FCF7F6FFF7
:10A380000AE0FDF703F807E00968C90606D430467D
:10A3900004E00EE0FDF70AF8002810D061684A08D2
:10A3A0001018FAF7A5FE80B201460E4A1039914204
:10A3B00003D9012503E01046F0E72168C8600020BA
:10A3C0006066A0662846F8BD00480040F369FFEFCC
:10A3D00000380140401002400044004000093D00A8
:10A3E000FFFC0F00EFFF0000F8B504464165403068
:10A3F00000262746028380373E602220E0672546FC
:10A40000206F603500281CD01749C162216F1748A2
:10A410000863216F16484863206F8663236F606D61
:10A420009C4613462168024660462431FCF726FA12
:10A43000002806D0102038602E752020A06701204B
:10A44000F8BD2E7520680168FF22013211430160BA
:10A450002068816801221143816020688168402260
:10A46000114381600020F8BDC9A0000827A10008A1
:10A470007DA00008FFB581B005460F460446603553
:10A480000A9E39E0701C37D0FCF7A0FB0499401AF3
:10A49000B04222D8002E20D02068016849072BD571
:10A4A000C069C043000527D401202168C0020862AA
:10A4B00020680168FF22A132914301602068816811
:10A4C0004908490081602020A067E067803420604F
:10A4D00000202875032005B0F0BD20680168FF2228
:10A4E000A132914301602068816849084900816078
:10A4F0002020A067E067EBE72068C1693846884301
:10A5000005D0002103988142BCD00020E3E701215F
:10A51000F8E7000010B504491020096808620248F5
:10A52000FDF704FC10BD0000CC16002001490D20F1
:10A53000887070475400002010B507480A22018A2D
:10A5400051430184FEF790F9FEF7A8FAC8220349A7
:10A550000348FDF79BFD10BD3C010020200D0020AD
:10A56000CC160020F8B53E4C002321783D4A1D460C
:10A57000082910D0072947D0062950D0052952D0E4
:10A58000042953D0032954D0002956D0012958D08A
:10A5900002295AD05BE0A17800264A1F04E0314F1F
:10A5A000BF5DFB189BB2761C9642F8DB6679277973
:10A5B0009A195118E3786278C9188918C91940188E
:10A5C000C0430006000E1AD1012E14D0022E16D15F
:10A5D00025482449C018FAF7D1FD01F02FFF642067
:10A5E00000F0A6FABFF34F8F21492048C860BFF39F
:10A5F0004F8F00BFFDE759081046FFF7A7F92570F8
:10A60000E570A570A571F8BDA1795054491CC8B278
:10A61000A071A178491F8842F5D1082001E060703F
:10A6200007202070F8BDE0700620FAE76071052071
:10A63000F7E7A070E5700420F3E7552807D1012063
:10A64000EFE7AA2803D10220EBE7032803D0257007
:10A65000E570A570F8BD032020702071F8BD0000E2
:10A6600034010020DE140020E80D00200400FA056B
:10A6700000ED00E010B5024A024900F0E5F910BD16
:10A6800031B80008880100202021020C01D01021DF
:10A690001046020A01D010460839020901D01046BE
:10A6A000091F820801D01046891E420801D0881E69
:10A6B0007047081A7047F8B5040C8BB2264682B270
:10A6C0005E430D0C1046370C5843360480190021A8
:10A6D000794116466E43370C360480197941264677
:10A6E0006E438919F8BD30B47446641E2578641C25
:10A6F000AB4200D21D46635D5B00E31830BC1847D7
:10A700004900CA020243100000D004204A0D01D0C3
:10A7100001221043044A490D914201D1022108430C
:10A72000012800D105207047FF0700008307FF22A2
:10A73000DB0E9A408907090E9940002808DB830840
:10A7400009489B001B18186890430843186070471D
:10A750000007000F0838830804489B001B18D869BD
:10A7600090430843D861704700E400E000ED00E04A
:10A77000BFF34F8F04490348C860BFF34F8F00BF3A
:10A78000FDE700000400FA0500ED00E0F8B504461E
:10A790004F1EC8000838211815461E46086849682B
:10A7A0003A4606239A4310D02A463346FAF76CFEFF
:10A7B0003A46D200083AA3181A687F1E5B68FAF777
:10A7C000B1FD06223B469343EED1022F23D0042F46
:10A7D00011D0062F2FD12A463346FAF755FEE36AE9
:10A7E000A26AFAF79FFD2A463346FAF74DFE636ADE
:10A7F000226AFAF797FD2A463346FAF745FEE369DF
:10A80000A269FAF78FFD2A463346FAF73DFE6369DF
:10A810002269FAF787FD2A463346FAF735FEE368E0
:10A82000A268FAF77FFD2A463346FAF72DFE6368E1
:10A830002268FAF777FDF8BD002210B513461046DE
:10A840000149FAF789FE10BD0000F03F10B5FAF794
:10A8500069FD10BD002210B5134610461146FAF7E7
:10A860007BFE10BD10B50721024A00200907FAF748
:10A87000EBFE10BD01030000034A10B500201107D4
:10A88000FAF7E2FE10BD000001FDFFFF02E008C87C
:10A89000121F08C1002AFAD170477047002001E05A
:10A8A00001C1121F002AFBD1704700000149086056
:10A8B000704700008C01002008B500216846017037
:10A8C0006B46012202212C2000F052FF0221684633
:10A8D00001706B4601222C2000F04AFF08BD0000E9
:10A8E00038B504466D20694608706B460122074959
:10A8F0002E2000F03DFF0649002C01D0054A00E063
:10A90000054A2E2000F01AFF38BD0000060800009E
:10A9100006180000070600000716000038B50446B8
:10A920006B4602220021362000F0EEFDB321230009
:10A93000FFF7D9FE0E0F08153A3A3A3A1C273A3A71
:10A940002F34483A00216846017040784108490098
:10A9500014E06946087880088000401C04E06946DD
:10A96000087880088000801C08701DE06846027826
:10A970000A404832027041788020014368464170A5
:10A9800012E0684602780A40027040784106490E9B
:10A99000F4E7694648780221084303E069464878AD
:10A9A000FD210840694648706B460122002136208F
:10A9B00000F0DEFE012200AB11463620013300F02C
:10A9C000D7FE38BD69460878CF2108406946203057
:10A9D000CAE708B5032168464170012101706B4642
:10A9E00002220021362000F0C3FE0122D2030621FC
:10A9F0002D2000F0A3FE012000F09AF80120FFF7BF
:10AA00008DFF08BD08B5020A69464A7008706B469A
:10AA1000022204212D2000F0ABFE032069460870BD
:10AA20006B46012206212D2000F0A2FE002069467F
:10AA300008706B46012206212D2000F099FE0A21A4
:10AA40002D2000F047FD08BDF8B516460F46044618
:10AA5000002503E03946B047641C6D1C20780028AF
:10AA6000F8D12846F8BD0000F8B54A002B4B520D2E
:10AA7000D6182B4A0C460546142E2BDA002E12DA75
:10AA8000284BFAF74FFC00221346FAF7A5FE40D2F6
:10AA9000002C03DA0124E40700253AE0204628438D
:10AAA00037D0214C14E0214F0B46F7403B402B435D
:10AAB00031D01C4BFAF736FC00221346FAF78CFE15
:10AAC00027D2002C03DD01200005F0400419BC430F
:10AAD00000251EE0332E1EDC33460027143BFF43C7
:10AAE000DF40384217D00F4BFAF7C6FC002213465E
:10AAF000FAF772FE0DD2002C0ADD142E0CD0342091
:10AB0000811B012088404019A84200D2641C0546E0
:10AB1000BD4321462846F8BD641CF9E701FCFFFF50
:10AB20009C7500883CE4377E0000F03FFFFF0F007B
:10AB30007D2110B5C900484300F001F810BD002187
:10AB400040E000BF00BF00BF00BF00BF00BF00BFAC
:10AB500000BF00BF00BF00BF00BF00BF00BF00BFFD
:10AB600000BF00BF00BF00BF00BF00BF00BF00BFED
:10AB700000BF00BF00BF00BF00BF00BF00BF00BFDD
:10AB800000BF00BF00BF00BF00BF00BF00BF00BFCD
:10AB900000BF00BF00BF00BF00BF00BF00BF00BFBD
:10ABA00000BF00BF00BF00BF00BF00BF00BF00BFAD
:10ABB00000BF00BF00BF00BF00BF00BF00BF00BF9D
:10ABC00000BF491C8142BCD37047FFB581B01E460F
:10ABD0000F46040026D00B9903980143A06A39431D
:10ABE000826807209047002818DB0A99A06A314341
:10ABF000826806209047002810DB25462035A97979
:10AC0000032F01D908200143032E01D90420014359
:10AC1000A06A826809209047002806DA0120C04314
:10AC200005B0F0BD0020C043FAE7384600F000F957
:10AC30002060304600F0FCF860600A986870039865
:10AC4000A870EF702E710B9868710020E8E7000083
:10AC5000F7B50446002090B000900190002C05D07C
:10AC60006A46062101F024FC062803DA0020C043CE
:10AC700013B0F0BD684640780102684600780004D1
:10AC80000918684680780818FAF71AFD05466846DC
:10AC90000391007901026846C078000409186846EB
:10ACA00040790818FAF70CFD032206460F46920772
:10ACB0005C4BFAF791FD07D200225B4B30463946D8
:10ACC000FAF7D4FB06460F4603229207554B284657
:10ACD0000399FAF781FD07D20022534B28460399C6
:10ACE000FAF7C4FB054603912068FAF7E9FC02462F
:10ACF0000B4630463946FAF72FFC07460A200791E3
:10AD0000205EFAF7C9FC3A46079BFAF7BDFB0646F8
:10AD100008200991205EFAF7ADFC0021C943FAF73B
:10AD2000F5FAFAF731FD3246099BFAF7FBFA06917C
:10AD300008906068FAF7C4FC02460B46284603995F
:10AD4000FAF70AFC05461A200E46205EFAF7A4FC24
:10AD50002A463346FAF798FB0C9009911620205E9C
:10AD6000FAF79AFC099B0C9AFAF7DCFA05910A901B
:10AD70002A46334638460799FAF786FB059B0A9A16
:10AD8000FAF782FB05910A901420205EFAF784FC02
:10AD90003A46079BFAF778FB07461C200791205E8E
:10ADA000FAF77AFC2A463346FAF76EFB0E900B91BF
:10ADB0001820205EFAF770FC0B9B0E9AFAF7B2FA95
:10ADC0002A463346FAF760FB0B910E902069FAF79A
:10ADD00063FC0B9B0E9AFAF7A5FA2A463346FAF75C
:10ADE00053FB05460E46E068FAF756FC2A46334602
:10ADF000FAF798FA3A46079BFAF794FA059B0A9AEB
:10AE0000FAF790FA01229207084BFAF73DFB024647
:10AE10000B46129C0898069903C411980CC0002098
:10AE200026E70000FFFF5F4100007041E17A843FA8
:10AE300000B50121C9040300FFF755FC081A0508F5
:10AE40000B0E1114171A0320C00400BD0720C00404
:10AE500000BD0F20C00400BD1F20400300BD3F20E7
:10AE6000400300BD7F20400300BDFF20400300BD24
:10AE7000084600BDFEB5264F0D4604000FD0002D3C
:10AE80000DD0264600202036B071F07129680D20C3
:10AE90008847002801DA7800FEBD102801D0384626
:10AEA000FEBDA562E968002901D028208847204618
:10AEB00000F030F80028F3DBA06AA52182680E209C
:10AEC0009047A06A962182680F209047A06A0221CD
:10AED000826862209047A06A002182680E20904715
:10AEE000A06A002182680F2090477179302001917B
:10AEF00000900623202201212046FFF766FE00284D
:10AF0000CEDB204600F0AEF80028C9DB0020FEBDF5
:10AF1000FFFFFFFF10B586B0044614216846FAF71C
:10AF200046F9002C7ED0A06A122143686A461020A0
:10AF30009847122877D168460078012201016846B7
:10AF4000407812030009081843492081884201DD36
:10AF5000801A20816846837840780007000D181811
:10AF60006081884201DD801A608168460079012293
:10AF700001016846C0781205000309186846407947
:10AF8000000908183549E060884201DD801AE06058
:10AF9000684640790007030B6846807900021B1859
:10AFA0006846C07918182061884201DD801A206146
:10AFB0006846417A007A0002081802B22848012146
:10AFC0000904A282824201DD521AA2826A46D37A21
:10AFD000927A12029A1812B2E282824201DD521A69
:10AFE000E2826A46537B127B12029A1812B22283C3
:10AFF000824201DD521A22836A46D37B927B12027F
:10B000009A1812B26283824201DD521A62836A4642
:10B01000537C127C12029A1812B2A283824204DD7F
:10B02000501A01E00BE008E0A083A06A0168282024
:10B030008847002806DA0120C04306B010BD002072
:10B04000C043FAE7C011C0072034002800D0802098
:10B0500060710020F1E70000FF070000FFFF07001C
:10B06000FF7F000010B5040009D0A06A07218268A4
:10B0700008209047002805DA0120C04310BD0020B9
:10B08000C04310BD072020342070002010BD0000F8
:10B09000FEB504460020019000906079734940009D
:10B0A0000E5A61782578491E7148CFB20163042D8C
:10B0B00077D0072D75D000210291217801736C495A
:10B0C000E379012292058969002B6CD0914381615B
:10B0D0006748217A4173217A82698907890B0A437B
:10B0E00082610021042000F034FB324661492E20A9
:10B0F00000F024FB3846FFF7F3FB5F4E0522705D3E
:10B10000810040185D49431807212B2000F030FBD7
:10B110005B49029801220B180B21282000F028FB24
:10B12000705D584980000A580C21282000F011FB5E
:10B13000E079554980004018A1794900425A02211E
:10B14000272000F0FBFA51487E00825B0421272073
:10B1500000F0F4FAE079002829D0A07804282CD057
:10B1600028206946087220220621272000F0E6FAEE
:10B1700002AB01222621272000F0FAFA44493801C7
:10B180004018E178890042580821272000F0E1FAB0
:10B19000A17A601C627A0902114313D016E000E024
:10B1A00001E0012188E71143F608816190E76422FC
:10B1B0000621272000F0C2FAE0E710206946087255
:10B1C0000246D1E733490172090A4172417A007A95
:10B1D0000A0202432021272000F0B0FA2E4F0C2152
:10B1E00023203A6800F0B5FAF01982880421232060
:10B1F00000F0A4FAA07900280BD0E07927490122B9
:10B2000043180021212000F0B3FA0320019001200F
:10B2100000902A07120F1001024360780021800776
:10B22000000B0243019800050243009840040243CA
:10B230002079C006400902436079C00602431F20FE
:10B2400000F087FAA07861780123084302040848D7
:10B25000DB030261E179490319430A4302610021DA
:10B26000082000F076FA0020FEBD0000E4C50008CA
:10B27000BC010020042800008CC500082400002028
:10B280004200002094C50008B4C50008C0C50008ED
:10B29000C4C5000841100000ACC5000844000020EF
:10B2A00038B50C4607498A8B002102432C2000F058
:10B2B00045FA684604706B46012206212C2000F0F6
:10B2C00057FA38BDBC01002010B5FFF7F5FA10BDE4
:10B2D00010B504460421362000F0FCF80121C90213
:10B2E000002C01D0084300E08843024604213620A8
:10B2F00000F02FFA10BD000038B5402069460870F4
:10B3000000210E2000F0E6F80446002211460E202F
:10B3100000F01FFA6B46012200210D2000F028FAF0
:10B32000074A00210F2000F014FA00F0EDF9224640
:10B3300000210E2000F00DFA02480021017338BDF3
:10B34000F8FF2724DC010020FEB5054604206946ED
:10B350000870514C002060752146203120634871EF
:10B360000873A0836063A06300F0C8F84B4E2060B0
:10B3700002E000F0C3F82060B042FAD10020FFF7ED
:10B38000CDFA00F0BBF8464E20603078242801D971
:10B39000243806E00621F9F7ABFE0622101A400118
:10B3A0000843020601040A4301020A430243B26051
:10B3B000706000211E2000F0CCF900F09FF82060A2
:10B3C0006B4601220021242000F0D2F91E20FFF755
:10B3D00019FB86B2300AA0730420FFF713FB07465F
:10B3E00000F08CF820603806000E0DD0022069466F
:10B3F000087101AB012212212D2000F0B9F9A08BB8
:10B40000012109030843A08300F078F8206006209A
:10B41000FFF7F8FA60600720FFF7F4FAA060F00683
:10B42000C00E207501D110202075C0B200F0DCF9EB
:10B43000E80707D0FFF7CDFAA08B0121C902084326
:10B44000A0830AE00521362000F02EF815490840B7
:10B4500002460521362000F071F90120FFF75EFA5F
:10B460000021042000F036F8A0610021262000F021
:10B4700031F815218903084302460021262000F0F7
:10B4800068F900222621362000F058F900F036F83D
:10B4900020600020FEBD0000BC0100203001CADE9B
:10B4A00018000020FFFD000038B5094C89B280B2B9
:10B4B0006B46022200F028F8002806D16846407842
:10B4C000010268460078081884B2204638BD0000A2
:10B4D000FFFF000038B50024E44389B280B26B4618
:10B4E000042200F011F8002806D103216846435CCD
:10B4F0002202D418491EFAD5204638BD10B50021C5
:10B500000846FFF7E7FF10BD38B5002909D04024F1
:10B5100020436C462070C8B27F2906D86070022094
:10B520000AE069460870012006E0802420436C464A
:10B530006070C809A0700320694600F059FF38BD4B
:10B5400010B5144603460A4621461120FFF7DCFFDA
:10B5500010BD10B50346052200211520FFF7D4FFCA
:10B5600010BD10B50346052200211720FFF7CCFFC0
:10B5700010BD38B5054600206946087000F0C4F8D3
:10B58000FF2401342246002D01D0032212020021A3
:10B590000D2000F0D3F8002D13D06B4601220321BB
:10B5A0000F20FFF7B1FF68460078000709D5FFF7C5
:10B5B000A3FE224600210D2000F0C0F80020C04369
:10B5C00038BD002038BD10B5024601210A2000F028
:10B5D000C0F810BD10B5044600211A20FFF77AFF0D
:10B5E000000D22030005120B024300211A2000F077
:10B5F000B0F810BD10B5024602492E2000F09EF8AA
:10B6000010BD000004180000F8B505466B46012285
:10B6100003210420FFF778FF0126114C3607002D87
:10B620000DD02A4600210C2000F088F869460878E1
:10B630001021084369460870A069304307E0694655
:10B640000878EF21084069460870A069B0430B46AE
:10B65000A06101220321042000F08AF8F8BD000057
:10B66000BC01002010B502460021182000F066F849
:10B6700010BD0000F8B50746002568460570B807FC
:10B68000204C2E4600280ADA8020694608706B4656
:10B69000012200210D2000F06BF801202073F80733
:10B6A0006946087821D006210843694608706B4630
:10B6B000012200210D2000F05BF803210F20FFF78D
:10B6C000F3FE8121C900084219D040206946087064
:10B6D0006B46012200210D2000F04AF80020FFF700
:10B6E000F7FD00252673ED4309E002210843694672
:10B6F00008706B46012200210D2000F039F8284621
:10B70000F8BD0000DC0100201CB56B4601220321BE
:10B710000F20FFF7F9FE684600784022C10910406B
:10B72000C9014000814208D00120694608710246E3
:10B7300001AB03210D2000F01BF81CBD08B56B46C2
:10B740001A70120A5A7089B280B2022200F010F800
:10B7500008BD38B500236C46E254120A5B1C042B6A
:10B76000FADB89B280B22346042200F001F838BD2A
:10B7700038B58024002909D0C02528436D4628709B
:10B78000C8B27F2907D86870022009E020436946C3
:10B790000870012004E020436870C809A8700320E5
:10B7A000694600F0CFFE38BD10B5144601231218CB
:10B7B0009B029A4202D90020C04310BD0B46821E54
:10B7C00021460920FFF7D4FF002010BD10B5054A1F
:10B7D0008905126901430A4300210820FFF7B9FFD8
:10B7E000002010BDBC01002038B504466B46012284
:10B7F0000E212B20FFF788FE68460078E1064009FD
:10B800004001C90E0143684601706B4601220E21BA
:10B810002B20FFF7ADFF38BD10B5002142541C06A8
:10B82000120A22431B0A491C0429F7DB10BD000041
:10B8300013B501231A4669460248FCF759FC0098E3
:10B840001CBD0000CC1600207CB5002425466846AF
:10B85000FFF77FFE04206946220E2D0215432202C7
:10B860000C5C1443401EF7D5204629467CBD7CB5B0
:10B87000002425466846FFF774FE04206946220E20
:10B880002D02154322020C5C1443401EF7D52046BE
:10B8900029467CBDFBF7A8F9FEF7F8F8FCF7F8FF9E
:10B8A00032493348002522C005608561C5613149B0
:10B8B0000562C1600838FBF707FBFCF7D5FFFDF711
:10B8C000EDF8FDF789F8FCF79BFF05260122360706
:10B8D000D1033046FBF773F9FDF788FEFCF788FECD
:10B8E000FAF75CF9FAF7DEF9FAF7ACF9FCF782FC43
:10B8F0000721B015FFF7D4FCFFF7E6FC1E4C0A2128
:10B90000208A01224843208411033046FBF757F96F
:10B910001748C8221949C830FCF7B8FB0126184F50
:10B920007603E07800281DD0607800281AD0E570F2
:10B9300020780F2802D9FEF7F7F90BE001223146F3
:10B940003846FBF73CF9FEF7EFF90022314638465E
:10B95000FBF735F9FCF772FD208C0028E1D0401E82
:10B960002084DEE7FCF76AFDDBE70000007C004096
:10B9700004160020FFFF00003C010020200D0020E5
:10B980000004005010B50122920217491748FAF737
:10B9900015FA1548164902888A4223D001800421ED
:10B9A0008180FF21F531C1800A21018100211E2201
:10B9B0004181D24382810122C28181834323C38694
:10B9C00002230387782343878287C2870246403257
:10B9D000118451849184C1839180142383821182C4
:10B9E00000F02CFD10BD0000E80D002000FC000858
:10B9F000AA550000F0B51FB496B084460C46024626
:10BA0000199D189803904900680063004908400890
:10BA10000193002A01D0012600E000269E19FE4B6A
:10BA2000F6185B109E422BD36E00039F0296002FE8
:10BA300000D00127F719F84EF84BBE199E421FD3CC
:10BA4000039E0346F64F334309D03B469C4201D147
:10BA5000002A04D0019B002A05D0012604E0002022
:10BA600039461BB0F0BD00269E19EE4B9E4207D80A
:10BA7000039F029E002F00D00127F6199E4207D98E
:10BA80002B4660462146189AFEF7E0FE1BB0F0BD3B
:10BA90000023002C29DAE44EB04226DAE34EB0420D
:10BAA00001DB022321E0DE4EB0421EDBE04E070D3B
:10BAB000BE19142E09DD3427BF1B039EFE400196DC
:10BAC000BE40039FBE420BD00FE0039F002F0CD15E
:10BAD0001427BF1B0646FE400196BE40864204D195
:10BAE000019BDE07F60F02239B1B0E46164318D15F
:10BAF000002D16DA002C03D0022B01D0012B06D02A
:10BB00000220FEF7D3FEFEF797FE1BB0F0BD022029
:10BB1000FEF7CCFEFEF790FE0122D20751401BB08B
:10BB2000F0BD039E002E61D1BF4EB04220D1C1486E
:10BB3000844201D1002A08D0B948814209DB002D96
:10BB400010DB189829461BB0F0BD0020B4491BB08B
:10BB5000F0BD002D06DA01222946D207189851407F
:10BB60001BB0F0BDB4497944086849681BB0F0BD0A
:10BB7000AB4FB84225D1002D1FDA002904D0B142C5
:10BB800012D1002A09D018E0002A72D1A649E20F8A
:10BB90000020D20711431BB0F0BD0020E20F014688
:10BBA000D20711431BB0F0BDB14206DA2346002094
:10BBB0003946F9F7D1FC1BB0F0BD104621461BB049
:10BBC000F0BDB14212DA0126B607B54203D12346D1
:10BBD00010461946FEE3994EB54207D1261E05DBF5
:10BBE0001046314600F040FC1BB0F0BD67007F08F6
:10BBF0001646002A40D100290AD08B4A914229D109
:10BC0000002C0EDD002D1CDB002011461BB0F0BD0A
:10BC1000022B16D0002C14D0012B12D1002C14DBD7
:10BC20000FE0002C28DA002D09DB012B03D00020C7
:10BC30007D491BB0F0BD002081491BB0F0BD012B38
:10BC400003D0002001461BB0F0BD00200121C90730
:10BC50001BB0F0BD724A91420ED1002C01DA002BCC
:10BC600017D0022B06D00020C043F9F715FD1BB0FA
:10BC7000F0BD90E20120F8E7E217521C94461A4307
:10BC800007D000220892664C62465B1E1A4307D01A
:10BC900009E00120FEF70AFEFEF7DCFD1BB0F0BD57
:10BCA0000022644C0892674A90427DDD664B674AE9
:10BCB00098421FDD914202DC002D05DB4DE0584823
:10BCC000814217DB002D48DD0220FEF7EFFDFEF775
:10BCD000C9FD05460E460022534B21460898F9F748
:10BCE000D3FB084671004908C00FC007014328462E
:10BCF0001BB0F0BD914215DA002D2EDA0220FEF7BE
:10BD0000D5FDFEF7AFFD05460E460022464B214607
:10BD10000898F9F7B9FB72005208C80FC007024330
:10BD2000114617E03E4B994223DD002D15DD022020
:10BD3000FEF7BCFDFEF796FD05460E4600223A4B87
:10BD400021460898F9F7A0FB084671004908C00F82
:10BD5000C007014328461BB0F0BD0220FEF7A6FD38
:10BD6000FEF78AFD49004908E20FD20711431BB0D4
:10BD7000F0BD002230463946F9F778FB012205462E
:10BD80000E46D243F9F760FC314A324BF9F774FBA7
:10BD90002A463346F9F778FB0022284BF9F76CFB6B
:10BDA00007462A46334600E064E0039110461946F0
:10BDB000F9F76AFB3A46039BF9F766FB074603224D
:10BDC00009915207244B28463146F9F75DFB07914C
:10BDD0000C90224A204B38460999F9F755FB074643
:10BDE00001911F4A1F4B28463146F9F74DFB3A4651
:10BDF000019BF9F73BFB07460B4602460991079961
:10BE00000C98F9F78FFA00250E462846079B0C9AE6
:10BE1000F9F72CFB3A4627E0FFFF1F00FFFF0F005A
:10BE20000000F03F0000E0FF0000F07F0000404312
:10BE300001FCFFFF0000F0BF560B00000000E03FD8
:10BE40000000F0FF0000E0410000F043FFFFEF3F83
:10BE5000555555555555D53F4715F73FFE822B652E
:10BE600044DF5DF80BAE543E099BF9F705FB024633
:10BE70000B4652E1012500202D05A94207DA3522A3
:10BE800030463946F9F7E0FB06463420C0430A1530
:10BE90001218FE48101803900803FD49000B0143D7
:10BEA0000F46FC49884201DC002003E0FA49884241
:10BEB00002DA0120119005E0002011900398401C47
:10BEC0007F1B039011980597C200F4480F927844A5
:10BED000801843680268394630460D930292F9F79C
:10BEE000C5FA07910C9030460D9B029A0599F9F717
:10BEF00019FA02460B460020E549F9F72DFB099196
:10BF00000490079B0C9AF9F7BFFA1290002010904A
:10BF1000E3480D46784400680E90012178104907E7
:10BF2000084311990D9B890440180121C904471841
:10BF30003946029A0E98F9F799FA3246059BF9F7B5
:10BF40009BFA02460B4629461098F9F79DFA0646D9
:10BF500002913B4629460E9A1098F9F795FA079BED
:10BF60000C9AF9F789FA3246029BF9F77FFA099B96
:10BF7000049AF9F789FA0591129A0A902B4610460D
:10BF80001946F9F781FA06460246C6480F460B469F
:10BF900006217844FEF7FAFB32463B4600910490B6
:10BFA00010461946F9F770FA009B049AF9F76CFAF3
:10BFB00006460F462B461946129A1098F9F7B2F921
:10BFC000059B0A9AF9F760FA32463B46F9F7AAF957
:10BFD000109A079104902B4610461946F9F754FA27
:10BFE000B14E0022334609910290F9F79BF9079B65
:10BFF000049AF9F797F90020074602463346009164
:10C00000F9F734FA099B029AF9F730FA079B049A78
:10C01000F9F732FA06460D913A462946009B1098E8
:10C02000F9F732FA07910C902B463046129A0D9987
:10C03000F9F72AFA05460E463A46009B05990A98F2
:10C04000F9F722FA33462A46F9F76CF902460B460D
:10C050000746099107990C98F9F764F900250E46EF
:10C060002846079B0C9AF9F701FA3A46099BF9F71B
:10C0700003FA07460722099152078C4B314628469E
:10C08000F9F702FA07910090894A884B38460999D6
:10C09000F9F7FAF907460191864A874B3146284657
:10C0A000F9F7F2F93A46019BF9F73CF9834B7B44E7
:10C0B0000F9A9B181A685B68F9F734F90290099196
:10C0C0000398F9F7E9FA05910490099B029A0799F8
:10C0D0000098F9F727F97A4B7B440F9A9B181A6856
:10C0E0005B6817460393F9F71DF9059B049AF9F766
:10C0F00019F90E462846059B049AF9F7B7F93A460E
:10C10000039BF9F7B3F9079B009AF9F7AFF9099B7D
:10C11000029AF9F7B1F902460B46199900200C90E2
:10C120000F461898F9F7B0F9029104903B460C9A23
:10C1300019991898F9F79AF92A463346F9F7A4F9A4
:10C14000029B049AF9F7EEF809910E902A463346BD
:10C1500039460C98F9F798F906460F46099B0E9A4E
:10C16000F9F7E0F8574A0D46914220DB5242AA18EF
:10C17000024310D132463B46F9F778F90490039117
:10C18000514A524B09990E98F9F7CCF8039B049A3F
:10C19000F9F722FB1ED20220FEF788FBFEF762FBB6
:10C1A00049004908E20FD20711431BB0F0BD6A00F5
:10C1B000474B52089A420DD3464AAA18024300D070
:10C1C000CBE532463B46F9F751F9099B0E9AF9F750
:10C1D00003FBF5D96800002340082C490393020DA6
:10C1E0003D4B5218984223DD01200005521CD040DF
:10C1F00042195000400D40183849794409681346E7
:10C200008C463749C1408B4312030121120B0905AB
:10C2100051181422101AC1400391002D01DA48422E
:10C220000390624630463946F9F720F906460F4634
:10C2300032463B4609990E98F9F774F800252A46CC
:10C24000284B28460591F9F71FF907910C90264ACB
:10C25000264B28460599F9F717F9009102903246C6
:10C260003B4628460599F9F701F9099B0E9AF9F71B
:10C2700003F91F4A1F4BF9F707F9009B029AF9F7D8
:10C2800051F807460B460246099135E001FCFFFFD5
:10C290000000F03F8E9803007AB60B00660700009E
:10C2A000A8070000D20600000000084009C7EE3FC2
:10C2B000FD033ADCF5015B14E02F3EBEA60500004D
:10C2C0006C05000000009040FE822B654715973CEE
:10C2D00000CC904000346F3F0000E03FC2040000FB
:10C2E000FFFF0F00432EE63F396CA80C615C20BEB7
:10C2F000EF39FAFE422EE63F07990C98F9F712F84B
:10C3000005460E46079B0C9AF9F7B0F83A46099B8A
:10C31000F9F7B2F809912A4633460E9010461946AD
:10C32000F9F7B2F8074602462F480B46059105215A
:10C330007844FEF72BFA3A46059BF9F7A5F82A460A
:10C340003346F9F799F80746019128463146099B8B
:10C350000E9AF9F799F8099B0E9AF8F7E3FF012373
:10C3600004910C9000229B0738460199F9F77EF85A
:10C3700005910E903A4628463146019BF9F784F81C
:10C38000059B0E9AF9F7E8F8049B0C9AF9F76EF8FA
:10C390002A463346F9F76AF80022144BF9F76CF88D
:10C3A000064603980D46000541190915002912DCBF
:10C3B00030462946039AF9F747F9FEF7A1F9042810
:10C3C00001D1FEF759FA30462946039AF9F73CF9AC
:10C3D000064601E004E029180B463246214608983B
:10C3E000F9F752F81BB0F0BD640300000000F03F05
:10C3F000F0B58C4600251026052109078E620E4CEB
:10C4000008E067467F5DE760A768FF07FCD0E76844
:10C410001F706D1C8542F4DB0020074606E0E760D4
:10C42000A568ED07FCD0E5681D54401C9042F6D38A
:10C430008E610020F0BD00000030014070B572B682
:10C440000124074DA40221462846F9F79DFC002847
:10C4500004D0224603492846F9F73AFD62B670BD7A
:10C4600000FC0008E80D0020F8B506460C46F9F778
:10C47000C1FA051E0F4600D00120014349000B48B8
:10C480004908411AC90F0DD0002E01D0012100E04A
:10C4900000210C4361004908401AC00F02D101205D
:10C4A000FEF704FA28463946F8BD00000000F07F88
:10C4B000F8B515460E460746002407E03819C0B205
:10C4C00000F008F8641C2870E4B26D1CB442F5D387
:10C4D0003046F8BD10B50446FBF74CFFEE20FBF7E5
:10C4E0001CFFFBF780FF2046FBF717FFFBF77BFFE6
:10C4F000FBF740FFEF20FBF710FFFBF774FF002076
:10C50000FBF7DEFE0446FBF750FF204610BD7047E8
:10C5100070B50D460446FBF72DFFEE20FBF7FDFE40
:10C52000FBF761FF2046FBF7F8FEFBF75CFF2846B0
:10C53000FBF7F3FEFBF757FFFBF737FF0A20FEF789
:10C54000FEFA70BDF0B50025102605279C463F0772
:10C550000B46BE620C4C06E0595DE160A168C9075C
:10C56000FCD0E1686D1C8542F6DB002007E06146E7
:10C57000095CE160A168C907FCD0E168401C9042F9
:10C58000F5D3BE610020F0BD003001400000010283
:10C5900003040005405C0000A05C0400C06C0800BF
:10C5A000805C0400E03F1E00E07D1E0007A902251C
:10C5B00070889B880A001600010006000100020036
:10C5C00087008D002D001A3152001A339A001A3557
:10C5D0001D011A376B003B31BE003B335E013B351A
:10C5E00096023B37000099599959EB518F421E45ED
:10C5F000142E0080EB51F5283333E13A703DE13AD7
:10C60000C235852BC2353333C235C235AE47E13A28
:10C610005138A33051380000000000000000010232
:10C62000030406070809030406080C10182030004C
:10C630000000000102030400000000000000F03FC1
:10C64000000000000000F83F0000000000000000B3
:10C650000000004003B8E23F0000000000000000BE
:10C6600006D0CF43EBFD4C3E033333333333E33F4C
:10C67000FFAB6FDBB66DDB3F4D268F515555D53F78
:10C6800001411DA96074D13F65DBC9934A86CD3F46
:10C69000EF4E454A287ECA3F3E5555555555C53F34
:10C6A00093BDBE166CC166BF2CDE25AF6A56113F26
:10C6B000F16BD2C541BDBBBED0A4BE726937663E28
:10C6C0000000000000000000E8C600080000002094
:10C6D00090010000BC5A00084CC7000890010020DF
:10C6E000681A00009CA800080124130704380D09EB
:10C6F0001E080540082609104008560A131D043B71
:10C7000008BE0516D8BC40100852010338C84205BF
:10C71000740CE5A00F1B0202DD140901022281F056
:10C720001F668104988996869679821598039814D5
:10C7300098879674977882439788967197778249FD
:0CC74000F10139293F9204922000000012
:04000005080050C1DE
:00000001FF
